:100000002EC4000054C4000052C4000050C40000BC
:100010004EC400004CC400004AC4000048C40000A4
:1000200046C4000044C400000C948D2E0C94762F1E
:100030000C94D80E3CC400003AC4000038C4000040
:1000400036C4000034C4000032C4000030C40000D4
:100050002EC400000C94692E2AC4000028C400009D
:1000600026C4000024C4000022C4000020C40000F4
:100070001EC400001CC400001AC4000018C4000004
:1000800016C4000014C4000012C4000010C4000014
:100090000EC400000CC400000AC4000008C4000024
:1000A00006C4000004C4000002C4000005010902E7
:1000B000A10185020901A1000509190129081500FE
:1000C0002501950875018102050109300931158165
:1000D000257F95027508810609381581257F9501D0
:1000E00075088106050C0A38021581257F95017572
:1000F000088106C0C005010980A101850319012AF4
:10010000B700150126B700950175108100C0050CD8
:100110000901A101850419012AA002150126A002E6
:10012000950175108100C005010906A1018506052C
:100130000719E029E71500250195087501810205D9
:1001400007190029EF1500250195F07501810205B9
:10015000081901290595057501910295017503910D
:1001600001C00660FF0961A1010962150026FF00B8
:100170009520750881020963150026FF00952075FA
:10018000089102C005010906A101050719E029E748
:1001900015002501950875018102950175088101F9
:1001A0000507190029FF150026FF0095067508812F
:1001B000000508190129051500250195057501910E
:1001C00002950175039101C041545A0041542B42DC
:1001D0004C45504F5745524C4556454C3D2D3132BC
:1001E0000041542B424C45484944454E3D31004165
:1001F000542B4741504445564E414D453D50616E4C
:1002000063616B650041542B474150494E54455240
:1002100056414C533D31302C33302C2C0041544549
:100220003D30004F4B0000000000000000000000C7
:1002300000000000000000000000000000000000BE
:10024000000000000000000000007E0F00D4FFFF4F
:10025000FFC70000007800000000000000002A2B0B
:100260002800000000000000000000000000000066
:100270000029000000002C1E3420212224342627CF
:10028000252E362D3738271E1F20212223242526F0
:100290003333362E37381F0405060708090A0B0CBE
:1002A0000D0E0F101112131415161718191A1B1C06
:1002B0001D2F3130232D350405060708090A0B0CC4
:1002C0000D0E0F101112131415161718191A1B1CE6
:1002D0001D2F3130354C09025B00030100A0FA09E3
:1002E0000400000103010100092111010001224461
:1002F0000007058103080001090401000203000052
:1003000000092111010001222200070582032000BB
:100310000107050303200001090402000103000096
:100320000009211101000122B60007058403200005
:1003300001120100020000000842534B500100016D
:100340000203011C037600690061006C003A00663C
:1003500000360034006300320062003300630000A6
:10036000001003500061006E00630061006B0065C7
:100370000000001203530070006100630065006D0F
:100380000061006E00000004030904290014001A33
:10039000000800150017001C0018000C00120013C4
:1003A000002A00225204001600070009000A000B70
:1003B000000D000E000F0033003400E1001D001B93
:1003C0000006001900050011001000360037003843
:1003D0000031002B002D002E00E300E0002C001E59
:1003E0007CE200215223522F0030000100D100CDC9
:1003F00000D2000100010001004B0052004E00013C
:100400000001000100CF00CE00D000010001004A31
:1004100000500051004F004D0001000100DD00DEE2
:1004200000DF0001000100010001000100010001E6
:1004300000010001000100010001000100010001B4
:10044000000100010001000100010035001E001F35
:100450000020002100220023002400250026002780
:100460000001000100010001000100010001000184
:100470000001000100010001000100010001000174
:100480000001000100010001000100010001000164
:100490000001000100010001000100010001000154
:1004A000000100010001000100010001003A003BD1
:1004B000003C003D003E003F004000410042004340
:1004C0000001000100010001000100010001000124
:1004D000000100010044004500010001000100018D
:1004E0000001000100010001000100010001000104
:1004F00000010001000100010001000100010001F4
:10050000000100010001000100007C41542B424C1D
:10051000454849444D4F555345425554544F4E3D1F
:100520000041542B424C454849444D4F5553454D8D
:100530004F56453D25642C25642C25642C256400EC
:1005400041542B424C45484944434F4E54524F4C22
:100550004B45593D3078253034780041542B424C7E
:10056000454B4559424F415244434F44453D253048
:1005700032782D30302D253032782D253032782DBF
:10058000253032782D253032782D253032782D25C2
:10059000303278001D020502EF01E101CC01C801F3
:1005A00041542B474150474554434F4E4E00415410
:1005B0002B4556454E54454E41424C453D307832D0
:1005C0000041542B4556454E54454E41424C453D05
:1005D0003078310001000100CD04D30D270E00005A
:1005E00002000200C904D30D270E00000300010021
:1005F000CE04D30D270E000004000200B304D30D77
:10060000270E020805000100CF04D30D270E0000BD
:1006100006000200B504D30D270E000007000200FB
:10062000CB04D30D270E000009000200B704D30D40
:10063000270E0B080A000200B904D30D270E0B0881
:100640000B000200BB04D30D270E0B080C000200A8
:10065000BD04D30D270E0B080D000200BF04D30DFF
:10066000270E0B080E000200C104D30D270E0B0845
:100670000F000200C304D30D270E0B081000020068
:10068000C504D30D270E0B0811000200C704D30DBB
:10069000270E0B0812000200D104D30D270E000014
:1006A00013000200D304D30D270E00001400010034
:1006B000D504D30D270E00001500000000003008FF
:1006C0006814000016000100D004EA0D3E0E000080
:1006D00017000101D004EA0D3E0E000018000102CF
:1006E000D004EA0D3E0E000019000200D704D30D1D
:1006F000270E00001A000103D004EA0D3E0E000090
:100700001B000200D904D30D270E0000FD377A58D4
:100710005A000004E6D6B44602002101160000008B
:10072000742FE5A3E001E900DE5D003D8889C65431
:1007300036C3174FE4F9EC72727025FA98E2F3FBB6
:100740007BF856EABCC9A0249B37CEA08A9152F30D
:10075000FC0745501339E17693723ABB304616D107
:100760004760E1B349F4E85186B1E42657ECBD6334
:10077000982B39BCB647DC6B258F09CDDACEED98C6
:10078000311F16F25FAB3E10A4FCD31A0A131240BD
:1007900021B45C94DEC9E50EF4A25AC452C1E2CE83
:1007A000E5914E5BE065BFBD5EF54E980893BF7165
:1007B0008FA72DC59D23D9C41FCDBDAF2C6EA673A9
:1007C000E79E74C39A34876EB0E6AF92106BEB82EB
:1007D000AF47216D447792915725C2E2B8C9CD0F3A
:1007E000D205B2ABD754B111729B481F196FBADB57
:1007F000C7DFCF00AE0AF8414F3A45173B2A2FA773
:1008000076922152BA374B7700000000CA551BAED2
:10081000EA6B6F960001FA01EA03000017D8B8F1FD
:10082000B1C467FB020000000004595A4C4C4C4C08
:100830004C4C2A52525252524C4C4C4C4C4C2A5218
:10084000525252524C4C4C4C4C4C2A5252525252D4
:100850004C4C4C4C4C4C005252525252CF0E112424
:100860001FBECFEFDAE0DEBFCDBF11E0A0E0B1E008
:10087000ECE8FAE602C005900D92AA3CB107D9F760
:1008800024E0AAECB1E001C01D92A23EB207E1F75C
:1008900014E0CFE2D4E004C02197FE010E945B3156
:1008A000CE32D107C9F70E94DD270C94DB34A8CBE8
:1008B0009C01FB019A9581159F4120F5832F817042
:1008C000B32FB270AA27732F74706627532F5870F6
:1008D000442734FF0DC08295807FAB2B09F08062E6
:1008E000672B09F08064452B09F08068099508950D
:1008F000AB2B09F08260672B09F08460452BB1F3C4
:100900008860F4CF80E0F2CF282F92959F709630C8
:1009100099F060F4925F9F70923030F4203FB1F014
:1009200038F481E0283E38F080E008959A5FF3CFF4
:1009300081E0243FC9F7089591E0813F09F090E0FC
:1009400081E0283E08F080E0892B089581E0089539
:1009500080936704089580936804089521E030E04F
:1009600001C0220F8A95EAF780916804822BF3CFA9
:1009700021E030E0A90102C0440F551F8A95E2F73B
:10098000CA018095909168048923E5CF292F94307E
:1009900090F58C3080F590E03CE0239F800D911D18
:1009A0001124282F277041E001C0440F2A95EAF74F
:1009B00023E0969587952A95E1F7FC01EE0FFF1F3E
:1009C000E80FF91FE75CFB4F20E030E070E0519149
:1009D000DF01CB01022E02C0969587950A94E2F7BB
:1009E000817081958527842385278E932F5F3F4FC4
:1009F0002330310561F70895292F943078F58C3034
:100A000068F590E03CE0239F800D911D1124682F34
:100A1000677023E0969587952A95E1F7FC01EE0F24
:100A2000FF1FE80FF91FE75CFB4F40E050E080E05C
:100A3000219130E0062E02C0369527950A94E2F700
:100A400021703327042E01C0220F0A94EAF7822B6B
:100A50004F5F5F4F4330510559F7089580E0089587
:100A60009091680421E030E0F90101C0EE0F8A9511
:100A7000EAF7D90102C0AA0FBB1F6A95E2F7EA2B79
:100A800001C0220F4A95EAF7892F8E23E81303C08D
:100A9000892F822B60CF2095822F8923FBCF8091D5
:100AA000380490E020E0022E001C000828170906F8
:100AB0000CF008952F5FF7CFFC01DB0184818130BA
:100AC00041F514968C911497813019F591818CE041
:100AD000E081F0E0899FE00DF11D1124E45DF74F06
:100AE00094919A32B1F011962C911197EC91F0E01B
:100AF000829FE00DF11D1124E45DF74FE49181E048
:100B00009E1301C080E091E0EA3209F090E0892B69
:100B1000089581E008959C01809169048D79811187
:100B200019C0211540E5340780F4211580E238070B
:100B3000C0F42333310511F1D0F481E02E313105B9
:100B400090F42430310530F00895C901965581158F
:100B5000914010F080E00895C901805F96450797A5
:100B6000C8F33327E6CF2C323105A1F70895265379
:100B7000310981E02330310538F3ECCF81E008956D
:100B80008091730490917204981301C008958F5F4F
:100B90008770FACF90916D048095892380936D04BE
:100BA000282F2770211110C0891771F09091DC0453
:100BB00092FF0AC0869586958695DADE10926D04BE
:100BC00010926F0410926E040895982F9095809162
:100BD00069048923809369040895809165048115CF
:100BE00031F0109265041092640410926304089529
:100BF000803E9105D9F1C8F48133910509F482C092
:100C000048F48932910509F472C08A32910509F4D9
:100C100080C0089589339105E9F082389105D1F0BB
:100C20008533910509F45EC00895843E9105D9F19C
:100C300048F4823E910539F1833E910549F181EEF8
:100C400090E00895863E9105C9F1873E910509F42B
:100C50003EC008952091DB042370211164C02091CF
:100C6000DC0423FF14C089E290E008952091DB04A6
:100C700020FD45C03091DC0430FF09C024FD24C0B4
:100C800083EE90E008952091DB0422FDF7CF0895D4
:100C90002091DB0422FD44C03091DC0430FD43C0D0
:100CA00024FFF5CF11C02091DC0421FFF0CF80910B
:100CB000DB0484FD09C087EE90E008952091DB04F9
:100CC00023FFE5CF24FFF7CF80E090E00895209147
:100CD000DB0423FD2BC03091DC0431FFE1CF84EE37
:100CE00090E008952091DB0425FFD1CFBCCF209167
:100CF000DB0425FD1EC02091DC0423FFC8CF89E35F
:100D000090E008952091DB0426FFC1CF8AE290E0B5
:100D100008952091DB0426FFBACF81E390E0089587
:100D200082EE90E0089580EE90E0089586EE90E0E7
:100D3000089585E390E008959091DB0492FF10C040
:100D400041E0282F2471243009F040E031E0282FC1
:100D50002871283009F030E0431711F02CE0822789
:100D600093FF10C041E0282F2471243109F040E0A6
:100D700031E0282F2871283109F030E0431711F0B5
:100D80002CE082273091DC0430FF10C051E0282F86
:100D90002171213009F050E041E0282F28712830DE
:100DA00009F040E0541711F029E0822731FF10C00C
:100DB00041E0282F2171213109F040E031E0282F56
:100DC0002871283109F030E0431711F029E082271B
:100DD00094FD877E08951F93CF93DF9309DFEC0185
:100DE000811522E5920708F052C0811540E594076D
:100DF00008F0CDC0803E910520F58D3C910508F0AE
:100E0000A1C0883A910570F4853A910508F097C021
:100E100081309105B9F10497813A910598F1C0E0CC
:100E2000D0E030C0885A91094B97C8F7C85AD0E033
:100E3000CC0FDD1FC55ADE4F0990D881C02DD46478
:100E400021C0811550E49507B0F4C11580E2D807A0
:100E500008F0B3C0C83ED105A8F0CE019A9581151F
:100E60009F41E8F68D2F68DF182FCE019927C0DE4D
:100E7000EC01D12B07C09927BBDECC27DF70C82B34
:100E8000D92BD06ACE01DF91CF911F910895803880
:100E900042E59407C8F5803652E5950708F05BC037
:100EA000C03482E5D807D0F4C03292E5D90708F003
:100EB0004BC08C2F8695869520E2829FC00111241D
:100EC000C37021E030E0A90102C0440F551FCA954C
:100ED000E2F7EA01C82BD92BDD68D4CF8C2F869599
:100EE0008695877050E2859FC0011124C37021E070
:100EF00030E0A90102C0440F551FCA95E2F7EA018C
:100F0000C82BD92BDC68BECF803C52E5950758F43E
:100F10008F71C03AD245A0F590E0982F8827EC0158
:100F2000C46FD06AAFCF805C9245809708F077CFCE
:100F3000DC2FCC27CC27DF71C06FD06AA3CFA4975A
:100F4000D064A0CFD0659ECFCF71D0E0DC2FCC276E
:100F5000C16FD06A97CF86958695877020E2829F71
:100F6000C0011124C37021E030E0A90102C0440F88
:100F7000551FCA95E2F7EA01C82BD92BDA6882CF50
:100F8000DBDEC82FD0E0DC2FCC27D0627BCF8F7187
:100F9000D3DE93E0CC0FDD1F9A95E1F7CC27DF700D
:100FA000282F30E084FF05C050E1859F9001112477
:100FB0003327C22BD32BD06965CF8D2F8F71BCDE29
:100FC000182FCE01992714DEEC01D12BDECF80E063
:100FD0000895F894E82FE295EF70F0E041A18F704A
:100FE00021E030E0B90102C0660F771F8A95E2F771
:100FF000CB01962F9095942391A392A1892B82A344
:10100000789408958091B3049091B4049093210151
:10101000809320010895E3EBF4E0848195812AE038
:1010200030E0B9010E9434316093240186818093BD
:101030002501828580930F01848580930E0186852A
:101040009785B9010E943431609322018089809391
:101050002301828980930D01848980930C01089576
:10106000EF92FF920F931F93CF93DF93FB018FEFCC
:101070009FEF4430510508F45FC04091DB0441FB11
:10108000882780F990E0880F991F42FB002700F91C
:1010900010E0000F111F000F111F802B912B40FB40
:1010A000EE24E0F8F12C8E299F2943FB222720F91A
:1010B000C22F50E0D52F53E0CC0FDD1F5A95E1F73A
:1010C0008C2B9D2B44FB222720F950E1259F90017A
:1010D0001124822B932B45FB222720F950E2259FD8
:1010E00090011124822B932B46FB222720F950E4F8
:1010F000259F90011124822B932B47FB222720F957
:1011000040E8249F90011124822B932B2091DC0432
:10111000322F3170932B26952170B22FBB0FA0E098
:101120008A2B9B2B092E000CAA0BBB0B808391836F
:10113000A283B38380E090E0CDB7DEB7E6E00C9405
:10114000253180E0089508950895AC0123E0969537
:1011500087952A95E1F78E719927FC01EB5EFD4F8B
:101160000190F081E02D4F70552721E030E002C062
:10117000220F331F4A95E2F7611541F0E22BF32B62
:101180008B5E9D4FDC01ED93FC9308952095309587
:10119000E223F323F5CF9091270198138093270141
:1011A00008958091E30087FD06C08091E4038111DA
:1011B00004C081E0089582E0089583E00895282F17
:1011C00035EB2303C001112497FF04C08058910917
:1011D000892F089580589F4FFBCF80914D046091D7
:1011E000BB047091BC0480FF14C020910F01269FA6
:1011F000C001279F900D1124BC01769567957695C7
:10120000679560387105F0F561157105E9F1862F74
:10121000089581FF0BC020910F01269FC001279FD9
:10122000900D1124BC0176956795EBCF82FF09C024
:1012300080910F019B01829FB001839F700D11244B
:10124000E0CF80914C048115E1F290910E01209144
:101250000F01891738F0CB01289FB001299F700D2D
:101260001124CFCF289F90011124269FA001279FF2
:10127000500D369F500D1124692F70E0CA010E9455
:101280003431BFCF8FE7089581E0089580914D04F8
:1012900080FF0CC060910D0170E0759567957595A4
:1012A00067956115710549F1862F089581FF06C084
:1012B00060910D0170E075956795F3CF60910D0118
:1012C00082FD0BC090914B049115A1F060910C012F
:1012D00080910D01961738F0682F70E06038710525
:1012E00000F38FE70895899FC001112470E00E94E8
:1012F0004831F4CF61E070E0D7CF81E0089580916C
:101300002701811101C04DDF813039F0833041F078
:101310008091D5039091D603089580E090E00895E0
:1013200080E091E0089580912701811101C039DFAB
:101330008D7F813029F081E090911201913009F088
:1013400080E00895DCDFFC01892B39F00190F08109
:10135000E02D309711F00995089580E00895A3E0FD
:10136000B0E0E5EBF9E00C940B318C0180911302B5
:101370009091140280179107A1F01093140200932A
:101380001302BDDFFC01892B61F00084F185E02DA3
:10139000309739F083E089831B830A83CE0101965D
:1013A00009952396E4E00C942731A3E0B0E0EBED3F
:1013B000F9E00C940B318C01809111029091120292
:1013C00080179107A1F0109312020093110297DF8A
:1013D000FC01892B61F00084F185E02D309739F014
:1013E00084E089831B830A83CE01019609952396A5
:1013F000E4E00C942731CF93C82F95DF811118C0FA
:10140000AEECB1E0EFEF80E09D91C91741F1EF3F05
:1014100019F4911101C0E82F8F5F8630A9F7EF3FD3
:10142000F1F00E2E000CFF0BE453FE4FC28317C0E9
:101430008091DB0487FFE4CFEC2FE695E695E695F7
:10144000C03F68F4F0E0EC52FE4FC77021E030E09E
:1014500001C0220FCA95EAF78281822B8283CF9145
:101460000895CF93C82F5FDF811521F08091DB04B1
:1014700087FD0CC0EEECF1E08191C81302C0DF01E2
:101480001E9281E0E43DF807B9F714C0EC2FE69511
:10149000E695E695C03F70F4F0E0EC52FE4FC77061
:1014A00081E090E001C0880FCA95EAF780959281AB
:1014B00089238283CF9108958091110108952FB7D8
:1014C000F89460910D0270910E0280910F0290913C
:1014D00010022FBF089587E797E790930108809344
:1014E000000888E19AE00FB6F894A8958093600010
:1014F0000FBE90936000FFCFFC019B01809103021F
:10150000909104028617970740F0672B29F4809189
:10151000E8008E778093E800C90140E0009741F42D
:10152000411106C08091E80082FF2FC080E008953D
:101530002091F9032115A9F12530A9F12091E800A6
:1015400023FD2DC02091E80022FDECCF2091E80082
:1015500020FFE4CF3091F3002091F200009719F0C2
:101560002830310558F041E02830310509F040E0DD
:101570002091E8002E772093E800D0CF419140934E
:10158000F10001972F5F3F4FE9CF8091F90381155B
:1015900041F0853041F08091E80083FFC3CF81E0C6
:1015A000089582E0089583E008958091FD0187FF0A
:1015B00013C08091E80082FF06C08091E8008B771D
:1015C0008093E80008958091F9038111F2CF089586
:1015D0008091F9038115D9F38091E80080FFF8CF5D
:1015E0008091E8008E77ECCF2091E4003091E50007
:1015F00095E6A9012091EC00822F817020FF06C0A2
:101600008091E80080FF06C080E008952091E80006
:1016100022FD1AC08091F903811589F0853089F087
:101620008091EB0085FD0FC02091E4003091E50032
:1016300042175307F9F29A95E1F684E0089582E0A3
:10164000089583E0089581E00895E8EDF0E0808159
:101650008E7F80831092E2001092DA001092E100F7
:10166000A0EEB0E08C9181608C9380818F77808335
:1016700019BCA7EDB0E08C918E7F8C9380818F7E1A
:1016800080831092FC010895CF93DF93D82FC92F48
:1016900036DEFC01892B49F00284F385E02D30977A
:1016A00021F060E28D2F9C2F0995DF91CF91089555
:1016B000982F9093E900891771F07091EC002091B8
:1016C000ED005091F00021FD09C09F5F973089F730
:1016D0008093E9000895762F242F50E03091EB009D
:1016E0003E7F3093EB003091ED003D7F3093ED0075
:1016F0003091EB0031603093EB007093EC0020935D
:10170000ED005093F0002091EE0027FDDECF08950C
:10171000A0E0B0E0EEE8FBE00C940731C8EDD0E0CB
:1017200088818F7E8883E7EDF0E08081816080830F
:1017300084E082BF81E08093FC0188818E7F888372
:1017400002EE10E0F80110821092DA0081EEC82E4D
:10175000D12CF601108288818F77888388818068F8
:10176000888388818F7D888319BC1092F903109239
:10177000FB011092FA011092F90190EEE92EF12C82
:10178000F70180818B7F808388818160888342E03C
:1017900060E080E08DDFF60180818E7F8083F8013C
:1017A000808181608083808188608083F70180816F
:1017B0008E7F8083888180618883CDB7DEB7E8E043
:1017C0000C942331E09173049091720427E0E913A3
:1017D00002C080E00895AE2FB0E02E9FF0011124EA
:1017E000EC58FB4F3181361306C03081381303C0EB
:1017F0003581341304C0FD013196E770E8CF81E0F4
:1018000008959C012115310509F408958FEC97E0A6
:101810000197F1F700C0000021503109F3CF0F9379
:101820001F93CF93DF938B01EA019091F9039430DA
:1018300051F58093E9008FEF9091E80095FD06C087
:101840009AE69A95F1F700C08A95B1F78091E80081
:1018500085FF19C0C9DE811111C08091E80085FDA6
:1018600006C08091E8008E778093E800F3CFF801FE
:1018700081918F018093F100219779F78091E800A1
:101880008E778093E800DF91CF911F910F9108959B
:10189000792F603229F440E250E0682F82E0BFCF18
:1018A0000895CF93DF93D82FC92F48E050E0682FD9
:1018B000792F81E0B4DF88E0ED2FFC2FA5E0B2E0C6
:1018C00001900D928A95E1F7DF91CF910895BC01C7
:1018D00040E250E084E0A3CFBC0146E050E084E069
:1018E0009ECFBC0143E050E084E099CF9091DC04AE
:1018F00092FB222720F9281771F080FB92F9909330
:10190000DC046091DB047091DC0484E090E00E94D0
:10191000C73482E03FC908953EDC6091270184E22C
:1019200090E00C94AD341F93CF93DF93962F122F3A
:10193000632F282F292B2430C8F44C30B8F4C42F3F
:10194000D0E0CC0FDD1F28E1929FC00DD11D1124E6
:1019500090E6899FC00DD11D1124CE0189960E9469
:10196000AD34612FCE018A960E94AD34DF91CF91C4
:101970001F9108950F931F93CF93DF9303EB14E010
:10198000C9EAD1E0CE010E949134F80161918F0142
:10199000681719F0CE010E94AD342196C13DF1E0E7
:1019A000DF0781F7DF91CF911F910F9108950F937A
:1019B0001F93CF93DF9303EB14E0C9EAD1E0CE018C
:1019C0000E949134F80181938F012196C13DF1E08D
:1019D000DF07A9F7CEEDD5E0FE018591959100973F
:1019E00011F0FC0109952C96F7E0C631DF07A1F74D
:1019F000DF91CF911F910F9108950F931F93CF9374
:101A0000DF93982F962B943020F54C3010F5C42F8F
:101A1000D0E0CC0FDD1F28E1629FC00DD11D112445
:101A200030E6839FC00DD11D1124CE0189960E94FE
:101A30009134082F10E0102F0027CE018A960E94C3
:101A400091349801282BC901DF91CF911F910F91FB
:101A5000089580E090E0F8CF462F672F2091FC0397
:101A60003091FD03232B81F4703F39F4403F61F442
:101A70008091FA039091FB030895982F972B94304F
:101A800018F44C3008F4B9CF80E090E00895A0E05D
:101A9000B0E0EDE4FDE00C9408317C0100916804B5
:101AA00080916704082BC3E0D0E010E0C8010C2E41
:101AB00002C0959587950A94E2F780FD09C02197A9
:101AC000A8F7D12C8D2DCDB7DEB7E7E00C942431EB
:101AD000DC2EB7018C2FC0DF7ED9019781F3F2CFC6
:101AE000CF93DF93D82FC92FD2DF6D2F7C2FB4DF98
:101AF00072D9DF91CF910895FC018481811529F07D
:101B000080819181EDDF0C94840480E008951F931F
:101B1000CF93DF93182FD92F611589F0411579F0F4
:101B2000B6DFC82F682F812F9D2F0E94C604612F1A
:101B30007D2F8C2F91DFDF91CF911F9108950E940F
:101B4000FC04C82FF4CFFC01462F65818081918170
:101B5000DECF382F292FCB01A32FB22F8F3222E0D7
:101B60009207A105B10520F48F529E4F0C94913439
:101B700080E0089585E290E00E949134853789F4F1
:101B800086E290E00E949134893059F487E290E037
:101B90000E94913491E0833309F090E0892F8170A5
:101BA000089580E0FCCF9C01CB01BA01F901329687
:101BB000E4914E2F50E06E17710548F0F90134960C
:101BC000659175910E94BC3180E090E008958FEF9F
:101BD0009FEF0895A4E0B0E0E0EFFDE00C940A313F
:101BE0008B01FC013396F49019821A821B821C82AD
:101BF000452B31F48FEF9FEF2496E5E00C942631CE
:101C000044E050E0BE016F5F7F4FCDDF019691F35E
:101C100081E090E00F2C02C0880F991F0A94E2F730
:101C2000092E000CAA0BBB0B49815A816B817C8168
:101C300084239523A623B72321E0892B8A2B8B2B82
:101C400009F420E0F801208380E090E0D5CF9C01EA
:101C5000CA01F9013296E4914E2F50E08E1791059A
:101C600050F0F9013496859195910E94BC3182DE45
:101C700080E090E008958FEF9FEF0895A4E0B0E03A
:101C8000E4E4FEE00C9406317C016B01CA01F7012B
:101C90003396B49019821A821B821C82892B31F4EC
:101CA0008FEF9FEF2496E9E00C94223144E050E05E
:101CB000BE016F5F7F4FC70176DF019689F381E038
:101CC00090E00B2C02C0880F991F0A94E2F78095D0
:101CD0009095092E000CAA0BBB0B49815A816B8190
:101CE0007C8184239523A623B723F6012081022F2C
:101CF000017010E00B2C02C0000F111F0A94E2F7D4
:101D0000012E000C220B330B802B912BA22BB32B1B
:101D100089839A83AB83BC8344E050E0BE016F5F4C
:101D20007F4FC70194DFBECFA0E1B0E0EAE9FEE05B
:101D30000C94FF30FE01319680E1DF011D928A95FF
:101D4000E9F703E210E091EDA92EBB24B3942FE252
:101D5000422E22E0522E612C712C4F017301620140
:101D6000B1E14B165104610471041CF080E1C82EEE
:101D7000D12CA601B501C4010E949E34AC0CBD1C3F
:101D80000D2C000CEE08FF084C185D086E087F084B
:101D90000150104019F76096E0E10C941B3110924D
:101DA000CB031092CC03E5E3F2E014821582089590
:101DB0001F921FB61F9211248F939F93AF93BF93CF
:101DC00080910D0290910E02A0910F02B09110022D
:101DD0004196A11DB11D80930D0290930E02A09318
:101DE0000F02B0931002BF91AF919F918F911F90FE
:101DF0001FBE1F9018952FB7F89480910D029091F7
:101E00000E02A0910F02B09110022FBF0895809191
:101E1000B5049091B604892B89F0EDDF209163041D
:101E200030916404AC01421B530B9A0181E0409154
:101E3000B5045091B6042417350708F480E00895DE
:101E4000CF93DF93C091690480916C04C82B80917B
:101E500065048115E9F08091B5049091B604892B51
:101E600021F0D5DF81110E94ED05D09165045BDA88
:101E7000811521F08091DB0487FD0EC086E02EECF9
:101E800031E090E0815060F491110E94ED05CD2B7E
:101E90008C2FDF91CF9108958EE126ED31E0F1CFC7
:101EA000F90141919F01411569F39F5FEBCF3BDA47
:101EB000811551F18091DB0487FF26C0C1DF80933B
:101EC000D50140E250E060E074E084ED91E00E94D2
:101ED000AF31892BC1F080E2E4EDF1E0A0E0B4E0A5
:101EE00001900D928A95E1F70ADAFC01892B59F0ED
:101EF0000480F581E02D309731F086E08093D401A5
:101F000084ED91E0099508959BDF8093CC0148E032
:101F100050E060E274E08CEC91E00E94AF31892BDC
:101F200091F388E0ECECF1E0A0E2B4E001900D92D6
:101F30008A95E1F7E4D9FC01892B29F30280F3812A
:101F4000E02D309701F38CEC91E0DCCF811531F07E
:101F500090916904892B80936904A9CF0895811514
:101F600031F090916C04892B80936C04A0CF08957C
:101F7000811519F00E94E5059ACF0895811539F071
:101F8000809590916C04892380936C0490CF089580
:101F900080912601877F8093260190916C049D7F1C
:101FA00090936C0484FF08C08F7E809326018091FB
:101FB00069048260809369048091260185FF08C0CE
:101FC0008F7D8093260180916904806280936904EB
:101FD0006ECF962F2091DC0422FF0FC0682F660F72
:101FE000660F660F692B60936D040E94AE0403DFD9
:101FF00090936F0480936E0408950C94AE049091B6
:102000006504292F2823211559F080958923809371
:102010006504811531F0EFDE8093630490936404CE
:10202000089580E090E0F8CFCF93C82F8091DC0432
:1020300082FF0BC0809165048C1739F0DCDE909331
:10204000640480936304C0936504CF910895EF9274
:10205000FF920F931F93CF93DF93EC018B0122E04C
:1020600030E040E060E084E30E945630C4DE7C0152
:1020700088810E9468308E3F9105E1F40E94CB3048
:1020800082E48A95F1F700C022E030E040E060E0B1
:1020900084E30E945630AFDE8E199F0980179107A6
:1020A00038F3C0E00E94CB308C2FCDB7DEB7E6E02E
:1020B0000C9425316B816F7770E06D5F7F4FCE019F
:1020C00001960E949830C1E0EDCFEF92FF920F93FE
:1020D0001F93CF93DF93EC017B018DDE8C0166991A
:1020E00022C082E08A95F1F700C085DE801B910B4B
:1020F0008E159F05A0F3C0E08C2FCDB7DEB7E6E0CC
:102100000C94253163E070E0CE0101960E94B1305D
:102110006B816F77613128F470E0CE0104960E94E4
:10212000B130C1E020C022E030E040E060E084E374
:102130000E9456300E94803088838E3F18F30E94A0
:10214000CB3082E48A95F1F700C022E030E040E035
:1021500060E084E30E9456304EDE801B910B8E15AA
:102160009F0540F3C0E00E94CB30C6CFA4E1B0E0B1
:10217000ECEBF0E10C940B31182FE0913A028091D6
:102180003902E81719F1669B25C066E970E0CE01B7
:1021900001969BDF8115D1F08C8187FD0DC02091C8
:1021A0003A0280913902281789F030E02F5F3F4FC3
:1021B0002170332720933A02111541F090913A0291
:1021C00080913902981711F06699DFCF6496E4E0A8
:1021D0000C942731F0E0EE0FFF1FEB5CFD4F008108
:1021E000118109DE801B910B8D32914078F3809133
:1021F0003A0290913902891749F390E00196817073
:10220000992780933A02E2CFF6DD20915004309175
:102210005104232B211521F08093E2039093E303D3
:102220002091520430915304232B211521F08093E7
:10223000E0039093E10363D8FC01892B59F00680F9
:10224000F781E02D309731F082E080934E048EE4E8
:1022500094E009950895611509F449C0E3E3E80F96
:10226000E33150F4F0E0E352FB4C0C945B310E94FC
:10227000ED08819580935104C7CF0E94ED08FACFF5
:102280000E94ED08819580935004F6CF0E94ED08DE
:10229000FACF0E94460980935204EECF0E9446096D
:1022A0008195F9CF0E944609819580935304E4CF2C
:1022B0000E944609FACF815D990B21E030E001C010
:1022C000220F8A95EAF780914F04822B80934F0466
:1022D000D3CF80914D04816080934D04CDCF809108
:1022E0004D048260F9CF80914D048460F5CF409118
:1022F00050048D3C59F48091510487FF0DC0109219
:102300005104411559F410924C0408C08E3C81F4DC
:102310008091510418169CF3411581F0809152046C
:1023200090915304892B8111A7CF10924B04A4CF15
:102330008F3C41F447FFF0CF10925004809151043C
:102340008115E0CF803D19F41416B4F3E5CF9091D8
:102350005204893D29F41916FCF610925204DCCF80
:102360008A3D19F497FFD8CFF8CF909153048B3D55
:1023700029F497FFD1CF10925304CECF8C3D19F49E
:102380001916CCF3C9CF9FE2980F983090F4815D75
:10239000990B21E030E0B90102C0660F771F8A95E2
:1023A000E2F7CB01809590914F04892380934F04ED
:1023B000B3CF8D3D31F480914D048E7F80934D04D9
:1023C000ABCF8E3D21F480914D048D7FF7CF8F3DB3
:1023D00009F0A2CF80914D048B7FF0CFCF93C82F0F
:1023E0008115A9F08CEF8C0F813A88F50E94930932
:1023F00081110FC0EEECF1E08191C81721F121E0CD
:10240000E43DF207C9F78C2F0E94FB0950DDCF9104
:1024100008958091DB0487FFEDCFEC2FE695E695DC
:10242000E695F0E0EC52FE4F828190E04C2F477031
:1024300021E030E002C0220F331F4A95E2F78223E9
:102440009323892B01F38C2F0CD831DDDCCF80E274
:102450008C0F883068F4C77081E090E001C0880F6D
:10246000CA95EAF7C0916904C82BC0936904CECF1E
:102470008BE58C0F833038F42C2F2452330BC90199
:102480000E94AF09C4CFE8E5EC0FEB3150F4F0E067
:10249000EE0FFF1FEF56FE4F808191810E94D509FC
:1024A000B6CF83E38C0F833108F0B1CF61E08C2F7E
:1024B000D2DEADCFCF93DF93EC01805E9109089718
:1024C00020F06FEA7FE0209711F466EA7FE0CE010A
:1024D0000E9458048C2F82DFDF91CF9108956115FF
:1024E00029F020916C04226020936C049C013052EE
:1024F0002115304308F49927DDCF811559F19CEF60
:10250000980F913A18F40E94310AD1CC90E2980FBA
:10251000983050F4877091E001C0990F8A95EAF7DE
:10252000892F0E94E505F1CF9BE5980F933020F4A9
:1025300080E090E00C94AF0998E5980F9B3120F46F
:1025400080E090E00C94D50993E3980F933110F458
:1025500060E081CE0895CF93DF93EC01CEDFCE0112
:10256000805E9109089720F06EEB7FE0209711F4D0
:1025700068EB7FE0CE010E945804DF91CF9108956F
:10258000CF92DF92FF920F931F93CF93DF93EC01D3
:102590008B01F42E8091260182FF61C0C090580407
:1025A000D0905904CC16DD0619F0209709F057C0D9
:1025B000809126018B7F80932601C1E081FD10C0B0
:1025C00080915604909157049801281B390BC1E063
:1025D00080912001909121012817390708F4C0E06B
:1025E00080912601C0FB81F9809326016C2FC601E2
:1025F0000E94A5088091690481FF08C0809126018E
:1026000080618093260182E00E94E5058091690443
:1026100085FF08C08091260180628093260180E2B8
:102620000E94E5056C2FC6015ADFF11431F080914C
:10263000CE0485FF02C086FF25C08091D104909111
:10264000D204DFD880915804909159049C013052F3
:102650002115304308F499277EDF9ADC0FC0CE01A4
:10266000905281159043B0F4CE01992774DF809188
:10267000580490915904C817D90779F31093570457
:1026800000935604DF91CF911F910F91FF90DF903F
:10269000CF900895CE01EACF1F93CF93DF93182FE9
:1026A000EB019CDE209731F4812F27DFDF91CF9162
:1026B0001F9108958FEC97E00197F1F700C000009B
:1026C0002197F0CF6091D3047091D404893321F025
:1026D0006091D1047091D204DFCFA0E0B0E0E3E7D5
:1026E000F3E10C940631EC0188818115D9F0813039
:1026F00009F03FC08981813021F48A812396E2DF8D
:10270000F3CF823021F48A81239668DEEDCF8330C7
:1027100021F48A812396F1DEE7CF843041F02296BE
:102720008111E2CFCDB7DEB7E9E00C9422318A8186
:10273000239620E030E09AE0682F6053770BAB01DE
:102740006A30710560F02115310551F3EFECF7E0C7
:102750003197F1F700C0000021503109F4CF929F6A
:10276000B001939F700D11249A01260F371F899194
:10277000E3CFE82FF0E0EA5AFD4FB490282F2695DA
:102780002695269530E0F901EA5BFD4FE4908770CD
:10279000F12C082E02C0F594E7940A94E2F7E0FACF
:1027A000EE24FF24E0F8F901EA5CFD4FC490D12C3F
:1027B000082E02C0D594C7940A94E2F7C0FACC243C
:1027C000DD24C0F8F901EA5DFD4F049110E002C07C
:1027D000159507958A95E2F701701127E114F10428
:1027E00011F081EEFBDDC114D10411F086EEF6DDAF
:1027F00060E070E08B2D50DFC114D10411F086EE43
:102800007CDEE114F10411F081EE77DE0115110593
:1028100011F08CE257DF219667CF109269040E9475
:102820009309811521F18091DB0487FF20C0E6ED3B
:10283000F1E08EE1DF011D928A95E9F780E090E0FA
:102840000E94AF0980E090E00E94D50910926C04CC
:102850002EDB86E0EEE4F4E0DF011D928A95E9F7D5
:1028600010924C0410924B0410924D04CDCCEEEC1F
:10287000F1E086E0DFCFD1DF2FE78AE196E021505B
:1028800080409040E1F700C0000088E19AE00FB678
:10289000F894A895809360000FBE90936000FFCFDE
:1028A000CF93DF93D82FC92F20913804283010F010
:1028B000B4DF20E0E22FF0E0EE0FFF1FE85DFB4FFA
:1028C000D083C1832F5F20933804DF91CF91089587
:1028D000CF93DF93FB018FEF9FEF44305105B0F0B2
:1028E000D081C1819ADFD093DB04C3708091DC0476
:1028F0008C7FC82BC093DC046091DB047091DC04F6
:1029000084E090E00E94C73480E090E0DF91CF91B6
:102910000895E3EBF4E0128E138E8FEA90E091833A
:10292000808325E0248F88E893E1938382838AE083
:1029300090E09583848344E150E05783468348E0E8
:1029400050E051874087938782876EE170E07587FA
:1029500064879787868780E590E0918B808B538B87
:10296000428B48E250E0558B448B42E350E0578B5A
:10297000468B48EC50E0518F408F158E55A344A3F1
:10298000178E168E91A380A322A317A216A20E94CF
:10299000BA0C43DF1092DC041092DB0480E0846008
:1029A0008093DC0460E074E084E090E00E94C7342F
:1029B0000C94D70C8F929F92AF92BF92CF92DF92DE
:1029C000FF920F931F93CF93DF938090F703909024
:1029D000F80381E090E09093F8038093F703A12C33
:1029E000B12C00E0650110E013C0FE012591359186
:1029F0004F2D612F802F0E94930C2296F3948CE030
:102A0000F812F3CF8CE0C80ED11C1F5F143039F0E0
:102A1000E601CC0FDD1FC557DC4FF12CE6CF0F5F71
:102A200080E3A80EB11C0430E9F673DF9092F8033E
:102A30008092F703DF91CF911F910F91FF90DF906C
:102A4000CF90BF90AF909F908F9008956FEF85E2E9
:102A500090E00E94AD346FEF86E290E00E94AD34CA
:102A60006FEF87E290E00E94AD3460E088E290E092
:102A70000E94AD349FDF58D965E785E290E00E945F
:102A8000AD3469E086E290E00E94AD3463E387E212
:102A900090E00C94AD34AAE2B0E0E1E5F5E10C94ED
:102AA0000C318DEF91E0FC0101962091F100208323
:102AB00022E085309207B9F78091FE01893009F450
:102AC00059C0C8F4823009F4B6C0833009F485C017
:102AD000813089F18091E80083FFEAC08091FD0197
:102AE0009091FE019A3008F0E3C0E92FF0E0E05148
:102AF000FB4C0C945B318A3009F48CC08B3051F75D
:102B00008091FD01813231F78091010290910202A2
:102B1000892B01F78091E800877F8093E8000E946D
:102B2000D50A81E09091FF01911101C080E080936E
:102B3000120173DECFCF8091FD01813A59F6809169
:102B4000E800877F8093E800809101029091020263
:102B5000892B61F060E080E090E070E00E947C0AE8
:102B60008091E8008B778093E800B4CF68E085E03F
:102B700092E0F3CF8091FD01813209F0ABCF8091DB
:102B80000102909102028D7F892B09F0A3CF8091E1
:102B9000E800877F8093E8008091E80082FF18C0FA
:102BA0009091F3008091F200029731F48091F1004E
:102BB000813011F0863021F48091F1008093110171
:102BC0008091E8008B778093E8000E94D50A82CF3D
:102BD0008091F9038111E0CF7DCF8091FD01813A91
:102BE00009F078CF8091010290910202892B09F0BF
:102BF00071CF8091E800877F8093E8008091E800A2
:102C000080FFFCCF809112018093F1008091E80059
:102C10008E77D9CF8091FD01813209F05BCF809111
:102C2000E800877F8093E8000E94D50A8091000227
:102C3000809310014FCF8091FD01813A09F04ACF76
:102C40008091E800877F8093E8008091E80080FF12
:102C5000FCCF80911001D8CF803889F0823841F5BF
:102C6000809101028F70873018F58093E900809180
:102C7000EB0085FB882780F91092E90006C080915F
:102C8000FA01880F9091F901892B9091E800977FC4
:102C90009093E8008093F1001092F1008091E80099
:102CA0008E7723C0811116C08091FF01813011F110
:102CB0008091E80083FF0AC08091E800877F8093BD
:102CC000E8008091EB0080628093EB00AA96E3E03D
:102CD0000C942831823061F78091FF01811589F0D1
:102CE0001092E9008091E800877F8093E8000E94BD
:102CF000D50ADECF81E0933009F080E08093FA01BD
:102D0000EFCF809101028F702FEF280F263080F6D1
:102D10008093E9002091EB0020FFE2CF933031F463
:102D20008091EB0080628093EB00DACF9091EB0012
:102D300090619093EB0021E030E0A90102C0440FC4
:102D4000551F8A95E2F74093EA001092EA008091BD
:102D5000EB008860E8CF8111ABCF1091FF011F77A6
:102D60008091E3008078812B8093E3008091E800DC
:102D7000877F8093E8000E94D50A8091E80080FF59
:102D8000FCCF8091E30080688093E30083E0111121
:102D900001C082E08093F9038BCF8058823008F025
:102DA00087CF8091FF01909100028C3D53E0950701
:102DB00099F583E08A838AE289834FB7F894DE012C
:102DC000139620E03EE051E2E32FF0E050935700ED
:102DD000849120FF03C082958F703F5F8F708A308F
:102DE000C8F0895C90E08D939D932F5F243161F74B
:102DF0004FBF8091E800877F8093E8006AE270E02F
:102E0000CE0101960E947C0A8091E8008B77809326
:102E1000E8004ECF805DE6CF292F332723303105E0
:102E200009F44EC078F52130310509F488C08BE5EE
:102E300090E0E6EDF2E02230310509F039CF209143
:102E4000E800277F2093E8002091030230910402DC
:102E50008217930708F49C0140E02115310509F021
:102E600073C0411171C08091E80082FDCDCF809187
:102E7000F903811549F2853039F28091E80083FF2A
:102E8000F2CFC2CF8091010290910202213231052E
:102E900009F446C02232310509F00ACF833091058A
:102EA00008F006CFFC01EE0FFF1FE15CFE4F019022
:102EB000F081E02D845C9E4FDC018C9190E010C08D
:102EC0009C013327823021F12330310568F4232B14
:102ED000B9F4E7E8F3E0E4918E2F90E0E7E8F3E05F
:102EE000009709F4E5CEABCF2330310509F0E0CEF1
:102EF000E3E4F3E0E4918E2F90E0E3E4F3E0F0CF3D
:102F0000E3E7F3E0E4918E2F90E0E3E7F3E0E8CF2E
:102F1000E1E6F3E0E4918E2F90E0E1E6F3E0E0CF2C
:102F20008330910508F0C4CEFC01EE0FFF1FEB5B70
:102F3000FE4F0190F081E02D89E090E080CF82E1AA
:102F400090E0E1E3F3E07BCF8091F903811509F490
:102F50005BCF853009F458CF8091E80083FD54CFD2
:102F60008091E80082FD7FCF8091E80080FF75CFDF
:102F70009091F3008091F2002115310519F088300D
:102F8000910550F041E0089709F040E08091E80099
:102F90008E778093E80061CF44914093F1003196A1
:102FA000215031090196E8CF803809F081CE809117
:102FB000E800877F8093E8008091FB018093F10017
:102FC0006DCE811175CE1091FF01123008F070CED8
:102FD0008091E800877F8093E8001093FB010E94B6
:102FE000D50A1115F9F084E08093F90342E061EC11
:102FF00081E00E94580B42E261EC84E00E94580B91
:1030000042E261EC82E00E94580B42E260EC83E015
:103010000E94580B8091F903843051F482E0809330
:10302000130146CE8091E30087FDDDCF81E0DCCF48
:1030300081E0F5CFEF92FF920F931F93CF93DF9331
:10304000C62FD42F122F8115A9F0609361040E941E
:10305000FB0E9093F8018093F701C77081E001C0E7
:10306000880FCA95EAF70E94A60FCDB7DEB7E6E053
:103070000C94253180916104681331C0E090F70110
:10308000F090F8010E94FB0E8E199F09883C910573
:1030900030F500E20D0FCD17A9F0C770FF24F394AF
:1030A0008F2D01C0880FCA95EAF70E94B80F08302B
:1030B00048F48D2F877001C0FF0C8A95EAF78F2D99
:1030C0000E94A60F812FFEDA083078F6D77081E0D3
:1030D00001C0880FDA95EAF70E94B80FC6CFC77013
:1030E00081E001C0880FCA95EAF7F6CFA8E0B0E00A
:1030F000ECE7F8E10C94FD308C01FC018481811532
:1031000009F4ACC260E0C8010E94A30D9C01F80163
:103110008681803170F44091730490917204491358
:1031200031C09091B104911521F09091B204903189
:1031300048F1F8019581911110C02115F0E53F0784
:1031400008F08AC0211540E2340708F09AC0283EF2
:10315000310588F4203E3105A8F4309355042093BE
:103160005404F801828193819093710480937004D8
:103170001092280107C0C9019A9581159F4168F7EF
:103180002111EBCF61E0C8010E94A30D7C01F80181
:103190008581811509F409C1C701975780389105C8
:1031A00008F003C1BE2CF0E1EF1608F047C26EE252
:1031B00072E080E090E00E94A90D81113FC2C12C15
:1031C000D12C7601B1105FC044E0242EAE014F5FD8
:1031D0005F4F58874F83EF81F885222D11922A95F2
:1031E000E9F7460157013FEF831A930AA30AB30A8E
:1031F000C701B6010E94A90D8983811509F41EC279
:10320000813009F0CEC02601370142E0440E511C46
:10321000611C711CC501B4010E94A90D382E8A835E
:10322000811509F40BC28FEF830D833008F040C085
:10323000C301B2010E94A90D8B83811519F0CE0143
:1032400001964BDA4601570153E0850E911CA11CF3
:10325000B11C75016401BFCF203E82E5380760F4E0
:10326000203892E5390708F08DCFC9018052924588
:10327000809708F072CF86CFC90187579C47029785
:10328000F8CF8031F6CF2FE2C21622E0D206E10459
:10329000F10409F4D3C1C701B6010E94A90D3FEFA3
:1032A000C31AD30AE30AF30A8111EDCFBA948ACF85
:1032B0008BEF830D8330F0F54601570183E0880ED4
:1032C000911CA11CB11CC301B2010E94A90D8B83EA
:1032D000811509F4BECFC501B4010E94A90D8C83EC
:1032E000811108C04601570194E0890E911CA11C70
:1032F000B11CAFCFAB80BC80E1E0AE16EFEFBE06F5
:1033000010F0BA2CAA24F6E03F1681F027E032161E
:1033100049F0C5010E9446248091D1049091D204C5
:103320000E94010CC5010E946724DCCFC5010E94E8
:103330004624D8CF34E05301420133128ACFC3016F
:10334000B2010E94A90D782E4601570144E0840E77
:10335000911CA11CB11CC701B6016D5F7F4F8F4F3F
:103360009F4F0E94A90D711409F468C1811509F4D9
:1033700065C18150990B4FEF489F9001499F300DD7
:103380001124E72DE150FF0B2E0F3F1F2150310973
:1033900008F45FCF8FEC97E00197F1F700C00000D1
:1033A000F5CFCE01019699D954CF8091CE0480FFFC
:1033B000BDC00E94FB0E5C01F8018581811509F4F6
:1033C000C6C08091260182FF05C040E0B50180E0C3
:1033D00090E0D6D8F4E1EF16FCE7FF0609F4B3C09D
:1033E00025E1E2162CE7F20609F44AC033E1E316C0
:1033F0003CE7F30609F48DC0C70190528115904354
:1034000008F048C01092590410925804F8019581B0
:10341000911110926104F6E1EF16FCE7FF0609F046
:1034200065C1809169043091CD0430FF04C0282F1C
:10343000247421114FC1282F2A7A31FF04C0482F4C
:103440004171411120E032FF04C0482F48784111FA
:1034500020E033FF03C08272811120E0911509F44E
:103460003BC181E0211101C080E08093620485E3CB
:10347000211101C089E20E94FB090E94570FDEC0A2
:1034800090912601892F8E7F90FF81608093260185
:103490000E94C80F8091260180FF48C0F8E2EF1615
:1034A000F10408F06CC02EE1E216F10408F07CC0D3
:1034B000C70104974A9790F58091CE0484FD2EC0F1
:1034C000F8018581811509F4E3C090916904809128
:1034D0006504D82ED92A2D2D2D7F211509F469C018
:1034E00010925904109258042091CE0421FD61C01D
:1034F00060E0C7010E94A50860E0C7010E946F124A
:10350000809165048D7F0E94141082E00E94CA059C
:1035100095C080912601816080932601F801858104
:10352000811521F01092590410925804F8018581F8
:10353000F701E851FC47E730F10508F067CFE650A6
:10354000FB4C0C945B31809126018E7F9FCF809144
:1035500026018F7E51EEE516F10439F085EEE8166E
:10356000F10431F4809126018F7D8093260192CF62
:10357000C70190528115904308F08CCF47CF39E3B3
:10358000E316F10468F44DE2E416F10420F45BE282
:10359000E516F10419F68091CE0482FDBFCF90CFDD
:1035A00084E6E816F104F6CF8091CE0483FDB6CF11
:1035B00087CF27E0F801AAE5B4E001900D922A95A3
:1035C000E1F710925D0410925C0480905804909092
:1035D0005904E814F90409F045C02091CE0425FFF0
:1035E00041C03091260131FBCC24C0F831FF02C02C
:1035F00026FF38C02091560430915704A501421B84
:10360000530B483C510570F591FF08C0809126018D
:1036100080618093260182E00E94E5058091690423
:1036200085FF08C08091260180628093260180E298
:103630000E94E5056C2DC4010E946F1280916D04FB
:103640008770811559F0F8018581811539F08091D5
:10365000DC0482FF03C082E00E94CA052896E2E1F2
:103660000C9419318D7F0E941410F0925904E0924D
:103670005804B0925704A09256048D2D8270846035
:1036800090912601997FD82ED92AD09226013DCF3C
:1036900040E0B501C7010E94C012D0CF26E241EE42
:1036A00061EEC8DCCBCF27E245EE65EEFACF26E22D
:1036B00041EE60EEF6CF27E245EE64EEF2CF26E271
:1036C00041EE62EEEECF27E245EE66EEEACF28E26B
:1036D00041E0EBCF20E0B1CE80916204811521F072
:1036E00085E30E94310AC9CE89E2FBCF27E7E216C3
:1036F0002CE7F20609F138E7E3163CE7F30639F167
:103700009701205E32452032310530F5911168C0B5
:103710004E2D4F7181E090E0FC0102C0EE0FFF1FC3
:103720004A95E2F77F016E2F83E090E00E94AD346E
:103730008E2D0E94A80482CF81E0911551F00E9445
:10374000AE0443E062E081E00E94300577CF82E082
:10375000F4CF0E94B804F5CF911509F458C0F701D1
:10376000E058F747E831F105A8F5EF5FFA4C0C9403
:103770005B3180912701E2E0811571F08230C9F060
:103780008330D1F0E0E008C0E0912701E11519F0A5
:10379000E230C1F7E1E0EF5FF0E0E953FE4F8081F6
:1037A0000E94CB086091270184E290E00E94AD3432
:1037B00045CFE1E0E150F0CFE2E0FCCF80E00E94B5
:1037C0008C0C3CCF81E0FBCF82E0F9CF83E0F7CFD8
:1037D00084E0F5CFFAE5EF16FCE7FF0609F499C09F
:1037E0002BE5E2162CE7F20608F06AC031E0E3169A
:1037F0003CE7F30609F48BC043E0E4164CE7F4061B
:1038000009F47FC0E1145CE7F50609F46DC0F80126
:103810008581C080D180811509F47FC0C6010E94D6
:10382000470DF82E682FC6010E94C604B6018F2DE1
:103830000E942C0D0E94EB06F82ED92E86E0F8018E
:10384000DE01119601900D928A95E1F7F801C5808D
:10385000B680B2942FE0B22280916D0487708115FA
:1038600009F1AC2CC114F9F0892F807F803469F004
:1038700080E28F0D8830B0F0892F807E803229F46D
:10388000F2E0FF1678F0B11469F08091DC0482FF59
:1038900009C082E00E94CA0580916D048770AA2445
:1038A000A3948111A12C8D2D82958F70882E912C3F
:1038B0008C3008F055C0F401E75EFA4C0C945B3193
:1038C0008BE5E8168CE7F80631F18091DC040024E2
:1038D00082FF0394802D9CE5E9169CE7F90609F028
:1038E00096CF0E94760C93CF0E940D14EFE7FAE179
:1038F00026E0E150F0402040E1F700C000000E94C7
:103900006B0A6FEF7FEF80E090E00E94C7340E9467
:103910003B1481E0E6CF80E0E4CFC6010E94FC04C6
:10392000F82E84CF2D2D2F70E22E30E1D31618F013
:10393000E29490EFE922C11409F44BC0E11469F05C
:1039400080E28F0D883010F0F1103DC08091690445
:103950008E29809369040E94570F8F2D0E94EE11CB
:1039600048E0841A910854E08516910418F40E94E6
:10397000A209A12C8F2D9D2D0E948404811541F058
:10398000C11409F425C2B11409F419C21092DF045C
:10399000A114A1F080916D0480FD10C0F801158282
:1039A0008695869586950E94AE04C8019FDB80911E
:1039B0006D048695869586950E94B80460E0C801DE
:1039C0000E94A30D4BCE80916C048E2980936C04D1
:1039D000C2CF8F2D0E947D12E11411F280E28F0D73
:1039E000883010F0F11004C08E2D0E94E50506C04D
:1039F000E09480916C048E2180936C040E94570F98
:103A0000AFCF8D2D8F70E82E8D2D807F803219F0F5
:103A1000E29480EFE822F11451F091E0F91609F4F4
:103A200075C0C11409F481C0B114E9F096CF80913A
:103A3000DC0482FD14C0C11459F0E11439F0809106
:103A400069048E29809369040E94570F80E086CF15
:103A500080E00E947D12E11409F482CFC5CFC11429
:103A600091F1B11004C08E2D0E94A60F79CFE1E034
:103A7000BE1211C0709065048E2D8721E81609F4DE
:103A80006FCF0E94FB0E90936404809363047E28A2
:103A90007092650465CF8091CF04823008F460CFC6
:103AA000B8125ECF8E2D0E94A60F8E2D0E94FF0FA2
:103AB000809166049E2D9823E91609F451CF8E2932
:103AC000809366044DCFB11012C08E2D0E94B80FA6
:103AD0008E2D0E94FF0F809166049E2D98239115D4
:103AE00009F43ECFE094E822E092660439CF809159
:103AF000CF04823008F434CFF1E0BF1231CF80918F
:103B000069048E21811509F42BCFDFCF8091D50474
:103B1000C11421F08B1508F423CFA5CFB81608F0F7
:103B20001FCF8E2D0E94B80F1BCFB114D1F329E304
:103B3000F21609F03CC18091D3049091D4040E9404
:103B4000010C8F2D0E947D120BCF8D2D86958695B1
:103B50008370811569F0813009F002CF8F2D9D2D82
:103B60009370C11002C080E090E00E94D509F8CEA9
:103B70008F2D9D2D9370C11002C080E090E00E94B7
:103B8000AF09EECE6C2D8F2D0E942B11E9CE8D2D1D
:103B90008370811133C0C110E3CE4F2D42954695FD
:103BA0004770440F440F8F2D8F70042E01C0880F73
:103BB0000A94EAF72F2D2071F4FE07C02FE030E0C1
:103BC00001C0220F4A95EAF720953D2D369536958E
:103BD0003370323071F0333051F04091670431303E
:103BE00029F0822B84230E94A804BACE842B822B36
:103BF000FACF822B909167048927F5CFC11459F130
:103C0000D0FEAECE4F2D429546954770440F440FDF
:103C10008F2D8F70042E01C0880F0A94EAF72F2D84
:103C20002071F4FE07C02FE030E001C0220F4A955A
:103C3000EAF720953D2D369536953370323091F068
:103C4000333071F040916804313049F0822B842385
:103C50000E94AB0485CE823008F482CED3CF842B71
:103C6000822BF6CF822B909168048927F1CF3D2DCE
:103C70003F70E32EC11429F0832F0E94AE048F2DD4
:103C8000F3CE8F2D0E94B80F8E2D0E94B80468CEFF
:103C900042EFF416A1F153EFF51670F480EFF81629
:103CA000D1F091EFF91691F0C11409F47BC0B11075
:103CB00054CE8D2D8F7127C0E3EFFE1639F1F4EF4E
:103CC000FF12F2CF8091DC0482FD2CC08D2D8F710C
:103CD000C114D9F218C08091D504C11461F0B8168E
:103CE00008F03ECE2D2D2F7181E090E001C0880FAD
:103CF0002A95EAF7B8CF8B1508F432CEF3CF8D2D85
:103D00008F71C110C2CF0E94AE042ACE80E0C114D0
:103D100009F49ECF81E09D2D9F7101C0880F9A9577
:103D2000EAF796CF8091CF04823048F1C114C9F0F0
:103D300090916D049770943059F410926D04109224
:103D40006F0410926E048D2D8F710E94B8040FCEF7
:103D500063E0B81608F00BCE8D2D8F710E94E90F2D
:103D600006CEB81640F010926D0410926F041092B7
:103D70006E0464E0F1CF81E00E94CA05F8CDC11461
:103D800031F063E08D2D8F710E94E90FE9CD81E064
:103D90000E94CA0522E0B21608F4E2CD82E00E9439
:103DA000CA05DECDB11441F039E3F316C2CE8091DD
:103DB000D1049091D204C3CE8D2D8F7166CF8091A6
:103DC0006B0480936A048091690480936B04E0CD56
:103DD00040E060E089819A810E94870D9C01E0901B
:103DE0006904B11429F01092DF04E0926B04D0CD85
:103DF0008091DD049091DE0428173907B1F7809196
:103E0000D00482FFF0CF8091DF04811561F38091AF
:103E10006A040E94A60F8F2D0E94621380916A048B
:103E20000E94B80FE0CF8091B204803178F4809185
:103E3000B104811559F0E09173042091720430911E
:103E4000AD044091AC0457E02E1301C008956E2FCD
:103E500070E05E9FF0011124DF01AC58BB4F149657
:103E60008C911497811551F111968C9111978313B0
:103E700025C08C91841322C015968C9115978111C1
:103E80001DC012968D919C91A091AE04B091AF048B
:103E90008A1B9B0B883C910588F48091B2048F703B
:103EA00080618093B204E658FB4F80818F708061FF
:103EB00080838CEA94E01AD90C94C005FB013196FA
:103EC000E770C2CFCF92DF92FF920F931F93CF93F1
:103ED000DF93182F092F87E0F82EC091730480918B
:103EE0007204C81791F1FC9EE0011124CE018C5898
:103EF0009B4F6C01FC018581811589F0C6010E94F0
:103F00007C0D811561F0FE01E658FB4F20812F707A
:103F100020612083F601808191810E945014C601A6
:103F2000E5D82091730430E02F5F3F4F277033278F
:103F300020937304CC58DB4F89818013CECF8881C6
:103F40008113CBCF8D81811541F2DF91CF911F91EC
:103F50000F91FF90DF90CF900895EF92FF921F9303
:103F6000CF93DF93EC0120912801211541F010E05F
:103F7000812FDF91CF911F91FF90EF900895EA80FC
:103F8000FB80E61AF70A24EFE21621E0F20678F742
:103F900060E0CE010E94A30D9C01305221153043F8
:103FA00030F70E948B05811511F380915404909194
:103FB00055040E948B05182F8115C9F28091D904F0
:103FC0009091DA04853F21E0920710F084EF91E0B0
:103FD000E816F90660F68E818F7080618E83888185
:103FE00099810E9450140E944F05CE017FD8C0CF06
:103FF000ADE0B0E0EEEFFFE10C94FF308C0186E025
:10400000F801DE01189601900D928A95E1F7D8012A
:104010006C9011965C9011971296AD90BC9013978E
:104020001496EC9014971596FC90F1100CC05091DA
:104030003804252F30E0E0E08E2F0E2E000C990B77
:10404000821793073CF15CEAC52E54E0D52E80918F
:10405000B004811151C0E114D1F0F11409F402C38C
:10406000C8010E947C0D811509F4FCC260917004A6
:1040700070917104C80171DF811109C087E0F801F6
:10408000ACEAB4E001900D928A95E1F7CCDEFF2412
:10409000F39486C0880F991F885D9B4FDC011196B1
:1040A0004C911197451103C08C91681611F0EF5F88
:1040B000C3CFEF3F41F2D80116968C9116978F70BF
:1040C000806116968C93E517A0F4AFEFA50FA0932F
:1040D0003804EA1770F4F0E0EE0FFF1FE85DFB4FC5
:1040E000B0E0AA0FBB1FA85DBB4F8D919C9191833F
:1040F00080830E944F05A7CF60E08CEA94E00E9485
:10410000A30D9C017090B1048091AE049091AF0416
:104110004501881A990A711409F451C2B8EC8B163A
:10412000910408F00AC2E11409F4B1CF8091AD0402
:10413000F8019181E090B204F0E1EF1608F0C6C1F9
:10414000981350C09091AC04D8018C9198134AC038
:10415000F11048C08E2D8F7080618093B2048CEA7C
:1041600094E00E9476188091B204F8018683F09062
:10417000AE04E090AF0447E0D42E00917304809128
:104180007204081751F0D09E800111240C581B4F67
:10419000D80115968C91811108C00E94C005F12CA0
:1041A0008F2D2D96E0E10C941B31F801B280C38075
:1041B000C8010E947C0D81110EC0C8010E947618B2
:1041C0008091730490E0019687709927809373041F
:1041D000FB2CEC2CD2CF6F2D7E2DC801BEDE8111C1
:1041E000EFCFDBCF30522115304308F084C0F110FF
:1041F00005C140E0652D862D0E94E20B81114FC064
:1042000040E0652D862D0E94E20BF82E811509F401
:1042100029C18091D00480FFC2CF8CEA94E00E9433
:10422000761860E08CEA94E00E94A30D8C01F09077
:1042300073047F2C98E0E92E2CEA822E24E0922E43
:1042400037E0432E809172047816A1F0A72CB12C90
:10425000479CC0011124FC01EC58FB4F6F0160E04A
:10426000CF010E94A30D582E692ED60115968C9170
:10427000811197C0B8E0EB1618F417E0EF10ACC04E
:10428000888599851FDE0E944F050E94C00587E042
:10429000ECEAF4E0DF011D928A95E9F780CF60E057
:1042A000C8010E94A30D8091D00483FFA9CFB8015B
:1042B0008CEA94E00E945C058111A2CF8091B20447
:1042C0008F7080618093B2048091AC049091AD04B2
:1042D0000E9450148CEA94E00E947618ECEAF4E014
:1042E00087E0DF011D928A95E9F788859985EADDE7
:1042F0000E944F0552CFF11409F482CF8091B2048D
:1043000081608093B2048091D00481FF48CF8CEA11
:1043100094E00E947618009173048091720408174B
:1043200009F4CCC0E02EF12CB7E00B9FC0011124A2
:10433000FC01EC58FB4F6F01CF010E947C0D8115F1
:1043400009F4BCC087E0F601ACEAB4E001900D923C
:104350008A95E1F7C701019687709927082F809306
:1043600073040E94C00587E0F82E809172048017C4
:1043700009F413CFF09E800111240C581B4FC80183
:104380000E947C0D811109CFC8010E94761880918E
:10439000730490E0019687709927082F8093730427
:1043A000E4CF10520115E0E31E0708F063CF8091BF
:1043B000D00483FD0AC0E72CC5010196F82FF770E1
:1043C0007F2E052D162D46013DCFB601C4010E945A
:1043D0005C05811589F3EFCF1F9DC00111248C5816
:1043E0009B4F0E9476182091730430E02F5F3F4F5F
:1043F00027703327F22E2093730440CF8091B204AC
:1044000081608093B20460E0C8010E94A30D809196
:10441000D00483FF78CFB8018CEA94E00E945C0559
:10442000811171CFF090B204E894F0F8F092B204E8
:10443000C8010E947C0D8111B2CE8F2D8F708061DA
:104440008093B2048091AC049091AD040E9450140A
:104450000E944F058CEA94E00E947618ECEAF4E0A2
:1044600087E018CF888599850E94700D292F2295A5
:104470002F70903450F49F70223080F0911599F095
:10448000F8019681903178F48BCE2A5F2F7022301C
:1044900078F0C8010E947618F72C82CE911519F099
:1044A000811509F47DCE805E883008F479CEF1CF95
:1044B000803F08F475CE815F8330F7CF87E0ECEA68
:1044C000F4E0DF011D928A95E9F74DCF981315C0EE
:1044D0009091AC04F801808198130FC0F1100DC0C9
:1044E000E682C8010E94761887E0F801ACEAB4E0E1
:1044F00001900D928A95E1F7CACDC8010E947C0D0A
:10450000811509F4AFC0F11409F4ACC08091B20474
:10451000803208F4B3CD8091AC049091AD049A83BD
:104520008983BC82AB828091B0048D831E82EF822E
:10453000CE0101960E947618A1CD9090B204F0E1D0
:104540009F1638F48CEA94E00E94761887E0D60132
:10455000A2CEE11409F49BCD9091AD04F8018181C4
:10456000981311C09091AC04808198130CC0F11085
:104570000AC09682C8010E94761887E0D6011D9273
:104580008A95E9F784CDC8010E947C0D811509F454
:1045900069C0F11409F466C08091B204803208F455
:1045A0006DCD8091AC049091AD049A838983BC82D7
:1045B000AB828091B0048D831E829F82B9CFB8EC0C
:1045C0008B16910408F052C0E11409F460CDF11487
:1045D00009F448C09091AD04F801818198132AC074
:1045E0009091AC048081981325C060E08CEA94E03F
:1045F0000E94A30D8091D7049091D8048816990643
:1046000008F072CF8091B20480FD6ECF803108F443
:104610006BCFD80116968C931697982F907F903F6A
:1046200009F45FCF982F907F905F8F70892B16963B
:104630008C9357CFC8010E947C0D811571F0609159
:10464000700470917104C80188DC811509F416CDDD
:1046500087E0ECEAF4E0DF0192CF8091B204816060
:104660008093B204C8010E94761811CD87E0F6014C
:1046700011928A95E9F793CDABE1B0E0E2E4F3E281
:104680000C9409314E8B5F8B688F798F082F8A8F3E
:10469000192F9B8FF82EE92E811509F4A1C040E057
:1046A000692F8E899F890E94870D9C01111549F001
:1046B0001092DF049093DE048093DD0410926C046A
:1046C0000AC08091DD049091DE048217930719F4EB
:1046D00081E08093DF041D8A86E0FE017696DE018C
:1046E0001F9601900D928A95E1F78091DC0482FF7C
:1046F00021C08091B5049091B604892BD9F00E9415
:10470000FB0E20916E0430916F04821B930B20915D
:10471000B5043091B6048217930738F080916D0488
:1047200082FD03C082E00E94CA050E94070F81112A
:104730000E94ED05F11461F00B8B1C8B61E0CE0142
:104740000F960E94A30D61E0CE010F960E94A30D6B
:104750000B8B1C8B87E0FE013F96DE0118960190C3
:104760000D928A95E1F7CE01089642DC811110C0C6
:10477000209172043091730487E0FE013896DE01C7
:10478000119601900D928A95E1F78C8581112CC0CC
:1047900017E08091730490917204891741F0189F7B
:1047A000C00111248C589B4F23DC811144C08C859F
:1047B000811112C08091280181110EC08A859B85CC
:1047C0002091700430917104821B930B8F3F9F43A3
:1047D00018F081E0809328016B96E6E00C94253177
:1047E000911509F478CF6ACF822F90E001968770F7
:1047F00099273817190671F40E940D14109272044B
:104800001092730487E0ECEAF4E0DF011D928A95D0
:10481000E9F7BECF97E0929FD0011124AC58BB4F6F
:10482000FE01319601900D929A95E1F78093720402
:104830000E94C005ADCF8091730490E0019687700F
:10484000992780937304A5CFA6E0B0E0EAE2F4E2F2
:104850000C940B310E94FB0E8C018091FE03909111
:10486000FF038017910771F019821A820E94FB0ED4
:10487000BC0149815A8180E090E0FEDE1093FF0385
:104880000093FE032696E4E00C942731A6E0B0E006
:10489000ECE4F4E20C940D319093FB038093FA0363
:1048A000811520E2920730F40E945A122696E2E027
:1048B0000C94293180EF89838A830E94FB0E8160EA
:1048C000BC0149815A8181E091E0D6DEEFCFA6E0BC
:1048D000B0E0EDE6F4E20C940D319093FB0380938D
:1048E000FA03811520E2920730F40E94AB1226965B
:1048F000E2E00C94293180EF89838A830E94FB0EC9
:104900008160BC0149815A8181E090E0B5DEEFCF42
:10491000A8E2B0E0EEE8F4E20C9400318C017B01F7
:104920005A014901FC0101900020E9F7CF010197EC
:104930006C01672BF1F590E1792E2AE0622E30E9C7
:10494000532EA601401B510B41315105DCF580E18E
:104950008D8B1E8A8AE08F8BCA018F779927888F6B
:104960005527B801CE0149960E94BC31B401CE0151
:1049700045960E942710182F8115B9F1E114F10412
:1049800009F047C00E94FB0EF82E092FE091390272
:10499000F0E09F012F5F3F4F2170332780913A0253
:1049A000821328C080E00E94B610F0CF81E00E9400
:1049B000B6109091390280913A029813F7CFF7011F
:1049C0001082B9CF7D8A1E8A6F8A588EF801DE0167
:1049D0005996872D01900D928A95E1F7B401CE0189
:1049E00045960E942710811102C010E00DC0005FA3
:1049F0001F4FA7CFEE0FFF1FEB5CFD4FF08201832F
:104A0000209339020E94FB0E812FA896EFE00C94B0
:104A10001C31AE0CBF1C87016CE271E0CE01019627
:104A20000E946510811509F38981803219F0F70120
:104A30001082DBCF8C818F77CA2CC01A8C1508F4BA
:104A4000C82EC11451F0D12CA601BE016B5F7F4F5F
:104A5000C8010E94BC310C0D1D1D8C8187FDDCCF6F
:104A6000F80110823197EE16FF0690F06AE070E0D0
:104A7000C7010E94D7319C01892B81F463E272E067
:104A8000C7010E948E3111E0892B09F4BDCFADCF53
:104A900080818A3031F38D3021F3E8CF2F5F3F4F93
:104AA0007901ECCFAAE7B0E0E8E5F5E20C94033138
:104AB0007C019091390280913A02981370C0409124
:104AC000CC038091CB03481709F469C08AE0849F26
:104AD000A0011124455C5D4FFA01DE01AF58BF4FC4
:104AE00001900D928A95E1F7FA01C0801581068147
:104AF000D780908481840E94FB0E9093E903809379
:104B0000E803F1E0CF1609F44FC022E0C21609F421
:104B100067C0C11036C06BE575E0CE0101965C013F
:104B20000E9497311F928F921F929F921F92DF9245
:104B30001F920F931F921F93E6968FADE6971F92D9
:104B40008F93E5968FADE5971F928F93BF92AF92AB
:104B50001F9280E38F938E010F5B1F4F1F930F9364
:104B60000E94E231970140E050E060E070E0C8014F
:104B7000CFDE0FB6F894DEBF0FBECDBF811509F4AE
:104B800099C08091CC039091CB03891741F090E0BC
:104B9000019668E270E00E9448318093CC03C658C9
:104BA000DF4FECE00C941F3160E475E08E010F5F85
:104BB0001F4FC8010E949731E6968FADE6978F93FD
:104BC000E5968FADE5978F931F930F931F9280E328
:104BD0008F93005C1F4F1F930F930E94E231C2CF4F
:104BE00061E275E0CE0101965C010E949731802F51
:104BF000002E000C990B9F930F93812F012E000C18
:104C0000990B9F931F93E6968FADE697282F082E5A
:104C1000000C330B3F938F93E5968FADE597282FCC
:104C2000082E000C330B3F938F93BF92AF921F92CD
:104C300080E38F938E010F5B1F4F1F930F930E9492
:104C4000E231970140E050E060E070E0C80160DED2
:104C50000FB6F894DEBF0FBECDBFB02EC12E8115AA
:104C600049F16BE075E0C8010E949731D0FE05C0A4
:104C70006BE271E0C8010E94CC31D1FE06C06DE24A
:104C800071E08B2D9C2D0E94CC316FE271E0D2FC43
:104C900004C0D11006C061E371E08B2D9C2D0E94F1
:104CA000CC31970140E050E060E070E08B2D9C2D0E
:104CB0002FDE64CFFFE729EA33E0F1502040304097
:104CC000E1F700C0000081E00E94B61068CFA0E0CC
:104CD000B0E0EDE6F6E20C940631FC01C080D28033
:104CE00003811481D581C681B78088E2E82EF12C3A
:104CF000E091CB038E2F90E00196B7010E944831DE
:104D00009091CC03981304C086E990E0CBDEF0CFFD
:104D10009AE0E99FF0011124E55CFD4F1082C38207
:104D2000D48205831683D783C087B1868093CB0353
:104D3000CDB7DEB7E9E00C942231A0E0B0E0E3EAC1
:104D4000F6E20C940831FC01E280F380D481C58145
:104D5000D18008E210E0E091CB038E2F90E0019625
:104D6000B8010E9448319091CC03981304C086E9A1
:104D700090E098DEF0CF9AE0E99FF0011124E55C25
:104D8000FD4F92E09083E382F482D583C683D7827D
:104D90008093CB03CDB7DEB7E7E00C9424310F93BB
:104DA0001F93CF93DF93FC018081843001F5C18193
:104DB000D28108E210E0E091CB038E2F90E00196C3
:104DC000B8010E9448319091CC03981304C086E941
:104DD00090E068DEF0CF9AE0E99FF0011124E55CF5
:104DE000FD4F91E09083D483C3838093CB03DF9105
:104DF000CF911F910F910895A2E0B0E0E2E0F7E2B9
:104E00000C9405318C017B016A012DB73EB73A83C2
:104E100029830E949E3101962DB73EB7281B390B7E
:104E20000FB6F8943EBF0FBE2DBF8DB79EB701964B
:104E30005C01B8010E94973126E930E0A601B70174
:104E4000C50166DD29813A810FB6F8943EBF0FBED9
:104E50002DBF2296EAE00C942131A8E0B0E0E3E314
:104E6000F7E20C940131FE01319688E0DF011D92DA
:104E70008A95E9F79BE4A92E91E0B92E8F013F01B5
:104E8000EE24E394F12C3BE5C32E31E0D32EF50163
:104E900081915F018F3F09F444C0F894E82FE295B7
:104EA000EF70F0E021A18F70A70102C0440F551FE1
:104EB0008A95E2F7CA01922F982B91A392A180952F
:104EC000892382A3789400C0EFE4F1E021E030E090
:104ED000812C912C41914F3F79F0A42FA295AF7076
:104EE000A05EB0E08C9190E04F7002C095958795E0
:104EF0004A95E2F780FF3BC080E090E0882A992A3B
:104F0000220F331FCE16DF0629F7F50182918F3F5E
:104F100011F00E94E90750E55A95F1F7D8018D92FA
:104F20009C920E5F1F4FBFE4AB16B1E0BB0609F0C9
:104F3000AECF48E050E0B3018DEC93E00E94AF317A
:104F4000892BB9F088E0F301ADECB3E001900D924C
:104F50008A95E1F781E08093F6010E94FB0E909321
:104F6000F5018093F4012896EEE00C941D31C901FF
:104F7000C5CF8091F6018115B1F30091F401109134
:104F8000F5010E94FB0E801B910B059760F348E032
:104F900050E06DEC73E08FEE93E00E94AF31892B0F
:104FA00049F088E0EDECF3E0AFEEB3E001900D9254
:104FB0008A95E1F71092F601D6CFCDB7DEB7CC587F
:104FC000D1090FB6F894DEBF0FBECDBF85B780689C
:104FD00085BF85B7806885BF84B7877F84BF0FB6DC
:104FE000F894A89580916000886180936000109289
:104FF00060000FBE80E890E00FB6F89480936100E7
:10500000909361000FBE81E08093130187EE97E0DB
:105010009093CB018093CA010E94D70C0E94250B6C
:105020000E94880B8091E20084608093E200789473
:105030008091F903811599F08091E9001091EC00BD
:105040008F70179511271795182B1092E9008091F2
:10505000E80083FD0E944B151F701093E90082E069
:1050600084BD93E095BD9DE797BD80936E000E943F
:10507000BA0D811102C00E94261585E30E94E9073E
:1050800087E90E94E90786E60E94E90780E90E9415
:10509000E9070FE411E0D8018D918D018F3F11F0E8
:1050A0000E94E907B1E00B351B07A9F788E0EFEE96
:1050B000F3E0DF01282F1D922A95E9F7EDECF3E0EC
:1050C000DF011D928A95E9F780E090E00E94993413
:1050D000833E9E4F21F40E94BA0D811130C063EED1
:1050E0007EEF80E090E00E94C73460E082E090E0D4
:1050F0000E94AD3481E08093670461E083E090E03A
:105100000E94AD3460E074E184E090E00E94C73416
:105110001092270160E084E290E00E94AD340E948A
:10512000261540E050E0BA018FE090E00E94BF34C5
:1051300040E050E0BA0183E190E00E94BF3482E099
:1051400090E00E9491348093D70384E090E00E9425
:1051500099349093DC048093DB047FDEEFE5FAEE74
:105160003197F1F700C0000078DE8091EF0380FFF7
:1051700008C06FEF7FEF80E090E00E94C7340E948C
:105180006B0A83E090E00E9491340E94A80484E2BC
:1051900090E00E9491348F3F09F483C080932701EF
:1051A0001092E5031092E6031092E4036E9876984D
:1051B000E8D6549A5C9A5C988FE19EE40197F1F7E7
:1051C00000C000005C9A9FEFA9E6B8E19150A040B2
:1051D000B040E1F700C0000081E08093E50384E186
:1051E00091E09093D6038093D5038E010F5F1F4FFC
:1051F00034DEF8ED6F2EF3E07F2EAFEEEA2EA3E063
:10520000FA2ED701F301219131918D919D9140EEBC
:1052100053E04E175F0709F44CC02817390799F37C
:10522000EFEE8E2EE3E09E2E312CD401CD90DD905A
:105230004D01F301419051903F014C145D0451F137
:105240004C245D24212CAA24A394B12CC2018A21D0
:105250009B21892BB1F029823A820E94FB0E9C830C
:105260008B83F1E0FD8391E096012A213B21232BE2
:1052700009F490E09E8349815A816B817C818D8104
:10528000FBD92394AA0CBB1C2CE02212DFCFF30124
:10529000D292C292339434E03312C7CF0E945F0A95
:1052A0000DC01092270160E084E290E00E94AD34CE
:1052B00077CF2817390709F0B3CFC6DA8091CE042B
:1052C00080FF1CC08091260182FF18C00E94FB0E47
:1052D000BC0180915604909157049B01281B390B07
:1052E00080912001909121012817390738F041E081
:1052F00080915804909159040E94C01286E0EEE417
:10530000F4E0D80101900D928A95E1F770904F0476
:1053100090905004A090510480905204B090530497
:10532000109250041092510410925204109253049F
:105330008A2D89298115A1F0C090E203D090E30362
:105340000E94FB0E9C012C193D0990914C04911573
:1053500009F4C1C0809125018217130608F4C9C061
:105360008B2D88298115A1F0C090E003D090E10336
:105370000E94FB0E9C012C193D0990914B04911544
:1053800009F4E7C0809123018217130608F4EFC0E7
:1053900080914F04781219C080915004811511F04A
:1053A000891113C020915104211511F02A110DC04B
:1053B00090915304911511F09B1107C03091520444
:1053C000311103C0822B892B81110E94041186E0C8
:1053D000F801AEE4B4E001900D928A95E1F7809176
:1053E000E6038111F4C08091E503811561F154E970
:1053F000C52E55E0D52E42E050E0B601CE018F57C4
:105400009F4F83D740E850E0B801CF57DF4F8881E6
:105410009981C158D040F0DC811589F0B2E0CB0E03
:10542000D11CE0EACE16E5E0DE0629F7F1E0F093C4
:10543000E6030E94FB0E9093E9038093E8038091BA
:10544000E6038111C4C00E94A2099091EA03891762
:1054500021F08093EA030E945F0A8091F90384306F
:1054600009F0C6CE43E04093E9008091E80082FF56
:10547000BFCE8091E80090E085FF0AC00E94F40A48
:1054800040E2A42EB12C6801811509F4EFC091E02F
:105490008091E8008B778093E800911509F4A8CEFD
:1054A000C090FC03D090FD03E981C114D10409F43C
:1054B000EBC0EE3F09F00BC18A81833020F08550AC
:1054C000833008F004C1EA81EE3008F000C1F0E05A
:1054D000EB5DFA4CF0C6409124018AE0849FA00164
:1054E00011244217530708F03BCF9F5F90934C0461
:1054F00002C09F3FD1F7911459F00E94ED0891E04E
:1055000019140CF09FEF899F802D11248093500473
:10551000A11459F00E94ED0891E01A140CF09FEFCD
:10552000899F802D1124809351048091500481150E
:1055300009F416CFD0905104D11409F411CF0E9470
:10554000DF08809350048D2D0E94DF088093510462
:1055500007CF40912201AAE0A49FA0011124421785
:10556000530708F015CF9F5F90934B0402C09F3FF5
:10557000D1F7811459F00E94460991E018140CF0FB
:105580009FEF899F802D112480935204B11459F00C
:105590000E94460991E01B140CF09FEF899F802D1B
:1055A00011248093530480915204811509F4F0CEA4
:1055B000D0905304D11409F4EBCE0E94DF088093FD
:1055C00052048D2D0E94DF0880935304E1CE81E0C8
:1055D0000E94B6108AE090E065DAC090E803D090AF
:1055E000E9030E94FB0E8C199D09893E934008F443
:1055F0002ACF8091E703811111C040E350E0B80148
:1056000081EC95E0F9DB811531F040E350E0B80121
:105610008EEA95E0F1DB31E03093E7030E94FB0E68
:105620009093E9038093E80340E350E0B80180EAF7
:1056300095E0E2DB811509F406CFC80149D69C014B
:1056400091E0232B09F490E08091E403981709F48A
:10565000FACE9093E403F7CE8091F100D6018D93BA
:105660006D01B1E0AB1AB10809F411CF8091E800E7
:1056700085FDF2CF8091E8008B778093E8000E944F
:10568000F40A811599F303CFE43148F4E11551F0A0
:10569000E150E33138F4F0E0ED5CFA4C0CC6EE3F3B
:1056A00009F411CFEFEFE98312C01A8289E08B83EE
:1056B0000EC08A81823079F08330B1F0813091F769
:1056C0000E945F0AFED56B837C838D839E83C80115
:1056D0000E94440B8DCD88E290E00E9491341B82A1
:1056E0001C821D828E83F3CF8091F7039091F80383
:1056F000892B69F3F80187EF93E0D7012C9111967C
:105700003C91B2E0EB0EF11C3283238332968E156E
:105710009F0599F7DCCF8A81823009F088C26B81BE
:105720007C818D819E81CDD588E290E00E94AD3450
:10573000CECF4C816B818A810E94FD0C98278927EE
:1057400098279E838D83C3CF2D813E8132272327C7
:1057500032274C816B818A810E94930CB8CF0E94C2
:10576000DA14B5CF80E18A83B2CF82E08A838FE2F8
:105770009ECF8C818D3108F0AACF8A809B8098249F
:1057800089249824A12CB12C78016801C80ED11C61
:10579000CE14DF0409F49BCF80E0FFE28F16F2E025
:1057A0009F06A104B10428F4C4018F529E4F0E94A9
:1057B0009134D70114968C93BFEFEB1AFB0AEFEFED
:1057C0008E1A9E0AAE0ABE0AE3CF8091F70390912B
:1057D000F803892B09F47BCF8C818D3108F077CFCA
:1057E000482E512C612C712CCA80DB80DC24CD2406
:1057F000DC24E12CF12C1801812C912C540184140F
:105800009504A604B70408F062CFFFE2CF16F2E0D9
:10581000DF06E104F10440F4D10114966C91C60155
:105820008F529E4F0E94AD34BFEF8B1A9B0AAB0A7A
:10583000BB0AEFEFCE1ADE0AEE0AFE0AFFEF2F1ABE
:105840003F0ADDCF0E94940E42CF84E08CCF8C8142
:105850008D3108F03CCF482E512C612C712CCA8020
:10586000DB80DC24CD24DC24E12CF12C812C912C58
:1058700054011E0125E0220E311C84149504A60457
:10588000B70408F024CF80E030E8C31631E0D30637
:10589000E104F10420F4C60189960E949134D101FB
:1058A0008D931D01BFEF8B1A9B0AAB0ABB0AEFEF6A
:1058B000CE1ADE0AEE0AFE0AE0CF2C81E22EF12C8F
:1058C0002D3108F004CF8A819B819827892798275A
:1058D0002C01612C712C8038F1E09F0708F0F7CE85
:1058E000822E912CA12CB12C40E851E060E070E0B8
:1058F0004419550966097709421751056105710573
:1059000008F4E5CE2091F7033091F803232B09F03A
:1059100053C09C01275D3F4FC557DF4F3983288314
:10592000CB58D04080FBCC24DD24C0F880FF0BC0D6
:105930008896F7D79D8189279827892781159C47C5
:1059400011F48FEF8D83D501C401840D951DA61D23
:10595000B71D80FF2AC0170141E0241A3108CE018B
:105960000596820D931DC757DF4F99838883C958C9
:10597000D040C557DF4F88819981CB58D0408E0DDC
:105980009F1DCFD7C757DF4FA881B981C958D040D5
:105990009C9181159C4741F48FEFC757DF4FE881F9
:1059A000F981C958D04080837101F801EC0DFD1DCB
:1059B0002FEFCE14DF0428F01801C12CD12C760172
:1059C00026C09481858181159C4711F42483258309
:1059D00042E0C40ED11C3296ECCF50E8451651E09F
:1059E00055066104710430F4D10114966C91C20122
:1059F0008996B3D7BFEFCB1ADB0AEB0AFB0AEFEFAE
:105A00004E1A5E0A6E0A7E0AFFEF2F1A3F0AC8146A
:105A1000D904EA04FB0408F35ACE8091F70390916D
:105A2000F803892B09F453CEC8010E94440B2FEFD1
:105A300030E742E0215030404040E1F700C0000034
:105A40009ECB88E0E3E3F1E0DE01AF57BF4F01906A
:105A50000D928A95E1F7FE0132968FE1DF011D92EA
:105A60008A95E9F786E0898388E0E158FF4FDE01F7
:105A7000159601900D928A95E1F729CE80E28983EF
:105A800081E08A831B821C8222CE8B819C81092E1D
:105A9000000CAA0BBB0B35E0880F991FAA1FBB1F78
:105AA0003A95D1F7AC01BD01405E5F4F6F4F7F4F1C
:105AB000481759076A077B0708F409CE8032E1E0EE
:105AC0009E07A105B10508F002CE4132F1E05F0763
:105AD0006105710520F040E251E060E070E0481B94
:105AE000590BBC01645F784FC8010FD4F0CD4AE177
:105AF00050E06FEF70E0CE01079647D48091F70336
:105B00008983CA821B821C821D828BE0EBCD81E0DF
:105B100090E09093FD038093FC0382E390E09093E8
:105B2000EE038093ED030E94FB0E9093EC038093B1
:105B3000EB03CDCDC114D10481F1B090EF03A0905F
:105B4000F003E090EB03F090EC030E94FB0E8E1943
:105B50009F098536910540F1A3FE26C0B0FE24C002
:105B60000E94FB0E9093EC038093EB038091ED0376
:105B70009091EE0301979093EE038093ED03892BB0
:105B800061F41092FD031092FC0381E090E0909389
:105B9000F8038093F703C12CD12C8091F7038983FC
:105BA000CA828091ED0383CD82E390E09093EE036F
:105BB0008093ED03F2CF1092F8031092F70387CD94
:105BC000EB80FC8040E250E06FEF70E0C801DDD375
:105BD00024ED35E042E050E080E090E0F90165918D
:105BE0007591E616F70630F4800F911FDC016D9376
:105BF0007C93CA01B7E020303B0709F468CDAC01C3
:105C00004E5F5F4F245F3F4F4132510538F35FCD08
:105C10002B813C8184ED95E0FC0145915591421723
:105C2000530759F10C96E7E08C309E07A9F78FEFE8
:105C300032C08B819C8124EDE22E25E0F22EF7010B
:105C4000259135918217930741F1FCE0EF0EF11C8D
:105C50002CE0E21627E0F20691F7CC24CA94DC2C63
:105C600036C00E94891433CD8B81811130CD80E202
:105C7000D8011D928A95E9F72ACDFC013696259127
:105C800035912115310599F24FE150E0BE016E5F6B
:105C90007F4FF901099589831ACDF701389625912F
:105CA000359121153105C9F24CE150E0BE016B5F21
:105CB0007F4FC701F90109956C01892B41F4F70168
:105CC0003A9685919591009711F0FC010995C9824A
:105CD000FECC78941F921FB61F9211248F939F932E
:105CE000AF93BF9380910D0290910E02A0910F028D
:105CF000B09110020196A11DB11D80930D029093E9
:105D00000E02A0930F02B0931002BF91AF919F912A
:105D10008F911F901FBE1F9018951F920F920FB664
:105D20000F9211242F933F934F935F936F937F9321
:105D30008F939F93AF93BF93EF93FF938091E10075
:105D400082FF09C08091E20082FF05C08091E100DE
:105D50008B7F8093E1008091DA0080FF23C08091E7
:105D6000D80080FF1FC08091DA008E7F8093DA0018
:105D70008091D90019BC80FFAAC082E089BD09B416
:105D800000FEFDCF81E08093F9038091FC01811139
:105D900009C00E94250B0E94880B8091E20084605C
:105DA0008093E2008091E10080FF1AC08091E200C0
:105DB00080FF16C08091E2008E7F8093E200809188
:105DC000E20080618093E2008091D800806280933D
:105DD000D80019BC85E08093F90383E08093130118
:105DE0008091E10084FF32C08091E20084FF2EC0E8
:105DF00019BC82E089BD09B400FEFDCF8091D800B6
:105E00008F7D8093D8008091E1008F7E8093E100A8
:105E10008091E2008F7E8093E2008091E2008160B9
:105E20008093E2008091FB01811509F455C084E064
:105E30008093F9030E940D140E94A2098091F90336
:105E4000843009F051C082E0809313018091E10019
:105E500083FF2CC08091E20083FF28C08091E10085
:105E6000877F8093E10082E08093F9031092FB0129
:105E70008091E1008E7F8093E1008091E2008E7F2F
:105E80008093E2008091E20080618093E20042E032
:105E900060E080E00E94580B8091F0008860809361
:105EA000F00081E08093130180931201FF91EF9144
:105EB000BF91AF919F918F917F916F915F914F9122
:105EC0003F912F910F900FBE0F901F901895109239
:105ED000F9031092FC0166CF8091E30087FF02C0B6
:105EE00083E0A6CF81E0A4CF81E0AECF1F920F92D6
:105EF0000FB60F921124EF92FF920F931F932F93DF
:105F00003F934F935F936F937F938F939F93AF9341
:105F1000BF93CF93EF93FF9309EE10E0F8018081D8
:105F2000C091EC008F70C795CC27C795C82B108205
:105F300080EFE82EF12CF7018081877F80837894B1
:105F40000E944B15F8011082F701808188608083E0
:105F5000CF70F801C083FF91EF91CF91BF91AF91C6
:105F60009F918F917F916F915F914F913F912F9171
:105F70001F910F91FF90EF900F900FBE0F901F9009
:105F80001895289A219A229A23982B9880E58CBDFF
:105F90000895FC0180912A018F3F09F085C080811E
:105FA0008F3F09F481C01092E1048181811519F0BD
:105FB00080E28093E10492818091E104923009F4BF
:105FC0004FC0933009F450C08460913009F449C047
:105FD0008381948121E030E02817390708F446C016
:105FE0008091E1042032310509F456C008F041C027
:105FF0002830310509F44BC02031310509F44AC07D
:106000002230310509F43FC08CB59091E104892B11
:106010008CBD8091E004811519F08DB581608DBD36
:10602000208120932A01458140932901E22FE295A6
:10603000EF70A1E2AE0FB0E03C912F7081E090E0F4
:1060400001C0880F2A95EAF7232F282B2C93EE5DA9
:10605000F0E09081411125C0892B808381E0089573
:1060600088608093E104B4CF8C60FBCF220F331F94
:10607000B3CF2034310599F083602038310521F603
:106080008093E104C1CF81E08093E004BDCF91E033
:106090009093E0048160F4CF91E09093E0048260FB
:1060A000EFCF80958923D9CF80E00895A6E0B0E0B6
:1060B000EBE5F0E3B2C089836A834B833D832C8395
:1060C00081E08E83CE01019664DF2696E2E0C1C0B6
:1060D000CF93DF938EBD0E94FB0EEC010DB407FE43
:1060E00005C08EB590E0DF91CF9108950E94FB0E20
:1060F0008C1B9D0B8436910588F38EEF9FEFF3CFB9
:10610000CF93DF931EBC0E94FB0EEC010DB407FE83
:1061100005C08EB590E0DF91CF9108950E94FB0EEF
:106120008C1B9D0B8436910588F38EEF9FEFF3CF88
:106130000F931F93CF93DF93EC018C01060F171F72
:10614000C017D10739F480E090E0DF91CF911F9123
:106150000F9108958991BCDF97FFF2CF8EEF9FEFEB
:10616000F4CF0F931F93CF93DF93EC018C01060FB5
:10617000171FC017D10739F480E090E0DF91CF916D
:106180001F910F910895BCDF97FD02C08993F1CF55
:106190008EEF9FEFF3CF20912A012F3F51F1E22F95
:1061A000E295EF70A1E2AE0FB0E03C912F7081E07C
:1061B00090E001C0880F2A95EAF7232F282B2C9313
:1061C000EE5DF0E0209129019081211599F0892B55
:1061D00080838FEF80932A018DB58E7F8DBD9CB516
:1061E0008091E104809589238CBD1092E104109286
:1061F000E004089580958923EBCF2F923F924F9230
:106200005F926F927F928F929F92AF92BF92CF9246
:10621000DF92EF92FF920F931F93CF93DF93CDB74F
:10622000DEB7CA1BDB0B0FB6F894DEBF0FBECDBFC7
:1062300009942A88398848885F846E847D848C8498
:106240009B84AA84B984C884DF80EE80FD800C81A1
:106250001B81AA81B981CE0FD11D0FB6F894DEBF84
:106260000FBECDBFED010895AA1BBB1B51E107C0B6
:10627000AA1FBB1FA617B70710F0A61BB70B881FD6
:10628000991F5A95A9F780959095BC01CD01089565
:1062900097FB072E16F4009406D077FD08D0E4DFB4
:1062A00007FC05D03EF4909581959F4F0895709519
:1062B00061957F4F0895EE0FFF1F0590F491E02D3B
:1062C00009946927962769277827872778270895CB
:1062D000FC0188279927E89421912032E9F329309D
:1062E00010F02E30C8F32B3239F02D3231F468948F
:1062F00003C02DD0820F911D219120532A30C8F365
:106300001EF4909581959F4F0895FB01DC0102C01A
:1063100005900D9241505040D8F70895FB01DC01E3
:106320008D91059080190110D9F3990B0895FB0107
:10633000DC0105900D920020E1F70895FC01059025
:106340000020E9F7809590958E0F9F1F08957AE0C1
:10635000979F902D879F802D910D11240895FB010B
:10636000DC0104C08D910190801921F4415050400E
:10637000C8F7881B990B0895FB01DC0102C001904E
:106380000D9241505040D8F70895DC0101C06D9343
:1063900041505040E0F70895FB01DC010D900020D2
:1063A000E9F7119701900D920020E1F70895FC01A3
:1063B00081E090E00190061609F4CF010020D1F7AA
:1063C00001970895AEE0B0E0E7EEF1E324CF0D8948
:1063D0001E8986E08C831A8309838F89988D81308A
:1063E00020E8920710F080E090E801979E838D836B
:1063F000AE01455E5F4F698D7A8DCE01019611D059
:106400004D815E8157FD0AC02F81388542175307A1
:106410000CF49A01020F131FF80110822E96E4E08B
:1064200016CFABE0B0E0E6E1F2E3EACE6C017B012F
:106430008A01FC0117821682838181FFCBC19AE019
:10644000592EF6012381F70123FD859123FF8191C8
:106450007F01811509F418C1853239F423FD959126
:1064600023FF91917F01953221F4B60190E0CBD1C9
:10647000E8CF30E0912C612C712CF0E27F1640F5D2
:106480009B32D9F058F49032D1F09332F1F09E3231
:1064900099F576FCF9C0689476F806C09D3291F0C3
:1064A0009033C1F4689470F8F70123FD959123FFB0
:1064B00091917F019111E1CF29C0689471F868949E
:1064C00072F8F2CF689473F8EFCF689474F8ECCF59
:1064D00077FC1CC080ED890F8A30C8F676FE05C0B7
:1064E000959C800D1124982EDFCF659C800D112482
:1064F000682E689475F8D8CF9C3619F4689477F8AC
:10650000D3CF9C3409F44AC0983671F2892F8F7D1D
:106510008554833008F444C0933609F464C093373B
:1065200009F467C0933509F472C0943619F09936AE
:1065300009F099C0F80177FE8FC061917191819146
:1065400091918F01272D2F76822E97FF09C090956C
:106550008095709561957F4F8F4F9F4F689487F816
:106560002AE030E0AE014F5F5F4F5A017CD18A19BB
:10657000A82E86FEBDC0882D8E7FA91408F0B7C056
:1065800084FE07C182FCFBC0F82DFE7E8F2EB92C45
:10659000882D8678811509F4B8C0F6C031E084CF23
:1065A0003115F1F0085F1F4F8FE3898388248394AE
:1065B000912CAE014F5F5F4F5A01E89477F873FC5E
:1065C00003C08614910498F181149104B1F561140B
:1065D00009F437CFB60180E290E015D16A94F7CF85
:1065E0000C5F1F4FE1CFF801808189830E5F1F4F41
:1065F000DDCFF801A190B1908F01692D70E076FC9C
:1066000002C06FEF7FEFC501F3D04C01D6CFF80188
:10661000A190B1908F01692D70E076FC02C06FEF00
:106620007FEFC501DAD04C01689477F8C8CFB60186
:1066300080E290E0E8D06A94C4CFF50177FC8591C0
:1066400077FE81915F01B60190E0DDD061106A9420
:10665000F1E08F1A9108B8CF61917191072E000C6B
:10666000880B990B6ECF872CE89484F82AE030E0F1
:10667000953731F1572D597F852E903791F050F491
:106680009835A1F09F36D1F0F601868197812B963F
:10669000EFE0D2CD9837C1F774FC05C020E130E0BF
:1066A0000FC0689484F8689482F8F8CF74FE03C031
:1066B000872D8660882E20E132E002C028E030E09D
:1066C000F80187FE0FC061917191819191918F01C5
:1066D000FE0131965F01AF01C6D08A19A82EE89459
:1066E00087F847CF6191719180E090E0F0CF882EDC
:1066F000BA2C84FE4DCFFE01EA0DF11D808180335E
:1067000009F040C0282D297E822E83FC0EC080FE19
:106710004BC09A2CB61418F4960C9B18B62C862DE8
:106720008B196B1408F480E0B80EB61408F03EC064
:106730006B1884FE3DC0B60180E390E064D082FE19
:1067400008C088E590E081FC02C088E790E0B601CF
:106750005AD0A914C8F1AA94B12C4FEFA41AB40AC4
:10676000CE0101964C01A80EB91EF50182915F0180
:10677000B60190E048D08A149B04B9F728CFB92C11
:10678000882EB9CF82FC02C0B394BFCFB394B39428
:10679000BCCFB92C882EFCCEB60180E290E033D07D
:1067A00073947614C8F3BBCF7B2CFBCF612CC1CF85
:1067B000882D8678811569F280E281FC8BE287FC66
:1067C0008DE2B60190E0C4CFB60180E390E01BD02B
:1067D0009A94BFCF8FEF9FEF5ACFFC010590615085
:1067E00070400110D8F7809590958E0F9F1F0895E7
:1067F000FC016150704001900110D8F78095909590
:106800008E0F9F1F08950F931F93CF93DF93182F21
:10681000092FEB018B8181FD09C01FEF0FEF812F45
:10682000902FDF91CF911F910F91089582FF14C097
:106830002E813F818C819D81281739073CF4E881A6
:10684000F981CF0101969983888310838E819F817E
:1068500001969F838E83E3CFE885F985812F099583
:10686000892BA1F3DACFFA01AA27283051F1203180
:1068700081F1E8946F936E7F6E5F7F4F8F4F9F4FD4
:10688000AF4FB1E03ED0B4E03CD0670F781F891F16
:106890009A1FA11D680F791F8A1F911DA11D6A0FE4
:1068A000711D811D911DA11D20D009F468943F9197
:1068B0002AE0269F11243019305D3193DEF6CF0196
:1068C0000895462F4770405D4193B3E00FD0C9F75C
:1068D000F6CF462F4F70405D4A3318F0495D31FDC9
:1068E0004052419302D0A9F7EACFB4E0A69597951C
:1068F000879577956795BA95C9F7009761057105F2
:1069000008959B01AC010A2E06945795479537953B
:106910002795BA95C9F7620F731F841F951FA01D95
:106920000895F999FECF92BD81BDF89A992780B557
:106930000895A8E1B0E042E050E02FC0DC01A40FD0
:10694000B51F4150504040F0CB01840F951F2E9150
:1069500005D041505040D8F70895262FF999FECF21
:1069600092BD81BDF89A019700B4021639F01FBAA2
:1069700020BD0FB6F894FA9AF99A0FBE08950396BF
:10698000272FECDFEADF252FE9DF242FE7CF019661
:10699000272FE4DFE2CFDC01CB01FC01F999FECF28
:1069A00006C0F2BDE1BDF89A319600B40D92415097
:1069B0005040B8F70895F894FFCF37113D114011BA
:1069C00046115B115B115B115B115B115B115B117C
:1069D0005B1149114E115211581169116F11731148
:1069E0002C165216581652165816AB16CD165816A7
:1069F000D417E117571B5B1B4E1B531B5F1B631BFD
:106A0000671BDE1BC41BB91BE21BE41BE81BE61B58
:106A1000EA1BEA1BEA1BEA1BEA1BEA1BEA1BEA1B4E
:106A2000EA1B1E1B1E1B1E1B1E1B1E1B1E1B1E1BD2
:106A30001E1B921C921C011D011DA51DC21DB01C18
:106A4000B01CC71D371E481E481E212D3E2D452D4A
:106A5000672B672B772D872D9A2DDB2DE02D082EA8
:106A6000192E312E342E552B592B8B2B992BA42BD1
:106A7000AF2B522B522B522B522B0D2DB22BB52B51
:0C6A8000B92BE52B222C252C272C5D2C9B
:106A8C00A1086726A3089D26CF26A40828081E0A5D
:106A9C00000001005C0A510C670C6C0C710C480C6A
:106AAC00AF000150011401FF0101FF4C0052004DD9
:106ABC00003000355BDCA2058C2C5C004422B684D3
:106ACC00016201AC00E8020103210335976690676F
:106ADC00963736F09293F1F4F5F6F7E200E900EA16
:106AEC0000B500B600B700CD008301CC008A01923E
:106AFC000194012102230224022502260227022AE4
:106B0C0002B300B4006F0070009F01CB019F02A084
:106B1C0002E200E900EA00B500B600B700CD008340
:106B2C0001CC008A01920194012102230224022546
:106B3C0002260227022A02B300B4006F0070009FE5
:0A6B4C0001CB019F02A0020002032A
:00000001FF
